:0400000007EF12F004
:1000080000C016F001C015F0E1CF17F0E2CF18F0EC
:100018009DAA65D09EAA63D0AECF24F3ABA20FD021
:10002800AB98AECF24F3AB88010E0201F425006E25
:10003800000EF521016E00C0F4F201C0F5F2ABA488
:100048000FD00201AB9EAB8E010EF425006E000EA0
:10005800F521016E00C0F4F201C0F5F2AECF24F331
:10006800030124510D0A07E02351000802E122513F
:100078007E0801E31ED0010E1E6F000E1F6F235174
:10008800000802E122517E0804E2020E1E6F000EF3
:100098001F6F9D9A2B0E2225E16E030E2321E26E1F
:1000A800E66A22C329F323C32AF3226B236B246B4A
:1000B80016D02B0E2225E16E030E2321E26E24C3F7
:1000C800E6FF22C329F323C32AF3010E2225006E7B
:1000D800000E2321016E00C022F301C023F39DA06E
:1000E8001ED09EA01CD00301010E255D006E000EDF
:1000F8002659016E00C025F301C026F3000E265DC7
:1001080002E1010E255D06E29D90CD90010E276F5C
:10011800000E286F3C0ECF6EB00ECE6E9E90F2A8E9
:1001280008D0F2A206D0010E0101816F000E826F85
:10013800F29216C000F015C001F017C0E1FF18C018
:04014800E2FF1100C1
:0C014C0072B201D0FDD71CC473FF12007A
:0E015800ACB202D00000FCD71CC4ADFF1200F8
:100166001BC404F08B94026A036A800E0318006EA7
:10017600800E005C02E1080E025C1FE2800E041491
:10018600016E0150800A02E18B8401D08B942A0E05
:100196000D6E0D2EFED70000043604908B802A0EBD
:1001A6000D6E0D2EFED700008B902A0E0D6E0D2EB5
:0C01B600FED70000024A032AD8D712002E
:1001C200086A096A100E0C6E0134083609360450AA
:1001D200085E0550D8A0053C095ED8B007D004508F
:1001E20008260550D8B0053C0926D89000360136BD
:0601F2000C2EEAD71200FA
:1001F800C7B409D01F0EC514016E0150000A03E1EF
:0A020800010E006E01D0006A120022
:10021200F250026EF29E0500FF6A0150FE6E00501F
:08022200FD6E02BEF28E120017
:10022A0014C400F00032009E0032009E0032009E8C
:10023A000032009E0A0E0002F3CF01F00F0E0401F5
:0A024A001415006E0150002612008A
:10025400F6C016F4F7C017F4F8C018F4F9C019F48E
:100264009E96C5869EB620D00001F651F711F8116E
:10027400F91119E0040116511711181119110CE1A3
:10028400E3C2E1FFE4C2E2FF030EE66EE1C200F066
:10029400E2C201F0BCDF08D0010E0401165F000EBB
:1002A400175B185B195BDED70401C9CF15F4145131
:1002B400000A02E1C58A01D0C59A9E96C588F6C097
:1002C40016F4F7C017F4F8C018F4F9C019F49EB680
:1002D40020D00001F651F711F811F91119E00401C9
:1002E40016511711181119110CE1E3C2E1FFE4C210
:1002F400E2FF030EE66EE1C200F0E2C201F087DF26
:1003040008D0010E0401165F000E175B185B195B21
:08031400DED715C400F0120051
:10031C00F6C014F4F7C015F4F8C016F4F9C017F4CD
:10032C00C582C5A220D00001F651F711F811F911C0
:10033C0019E0040114511511161117110CE1E3C247
:10034C00E1FFE4C2E2FF060EE66EE1C200F0E2C29B
:10035C0001F059DF08D0010E0401145F000E155B8B
:08036C00165B175BDED71200DF
:100374000B6A0A6A096A00500402F4CF09F0F3CF49
:1003840008F001500502F4CF0BF0F3CF0AF000504F
:100394000502F3500926F4500A22E86A0B220150A0
:1003A4000402F3500926F4500A22E86A0B2208C01A
:1003B40000F009C001F00AC002F00BC003F0120003
:1003C4008B924F0E0D6E0D2EFED70000000081A6FD
:1003D40019D014C41BF4C5DE18C41BF4C2DE14C443
:1003E4001BF4BFDE17C41BF4BCDE14C41BF4B9DE5B
:1003F40016C41BF4B6DE14C41BF4B3DE15C41BF41C
:10040400B0DE18D014C41BF4ACDE15C41BF4A9DE92
:1004140014C41BF4A6DE16C41BF4A3DE14C41BF41C
:10042400A0DE17C41BF49DDE14C41BF49ADE18C4AA
:100434001BF497DE350E0D6E0D2EFED78B82120047
:04044400C584120059
:080448000AAE029E000E120034
:100450000B840BAE33EF02F0010E036E026A016AE9
:0A046000006A0A360232FF0E120095
:0E046A00026A016A006A086A036A000E120044
:100478009E9614C4C9FFF6C015F4F7C016F4F8C068
:1004880017F4F9C018F4C7A422D00001F651F711E7
:10049800F811F9111BE00401155116111711181163
:1004A8000EE1E3C2E1FFE4C2E2FF040EE66EE1C240
:1004B80000F0E2C201F0A9DE010E006E3BD0010E91
:1004C8000401155F000E165B175B185BDCD7F6C0DE
:1004D80015F4F7C016F4F8C017F4F9C018F49EB66E
:1004E80022D00001F651F711F811F9111BE00401AF
:1004F80015511611171118110EE1E3C2E1FFE4C2FC
:10050800E2FF040EE66EE1C200F0E2C201F07DDE19
:10051800010E006E0FD0010E0401155F000E165B70
:10052800175B185BDCD7C5BC02D0006A03D0C58452
:06053800020E006E12002D
:10053E00086A080E0C6E003408360450085ED8B0F7
:0E054E0002D00826D89000360C2EF5D71200E9
:10055C00F6C016F4F7C017F4F8C018F4F9C019F483
:10056C000401146B156B1551120802E114518E081D
:10057C0008E33CDE005201E004D00401144B152BBF
:10058C00F2D70401120E155D02E18F0E145D03E328
:10059C007B0E006E26D0C580C5A022D00001F6517E
:1005AC00F711F811F9111BE004011651171118116C
:1005BC0019110EE1E3C2E1FFE4C2E2FF050EE66EA3
:1005CC00E1C200F0E2C201F01EDE010E006E09D0A5
:1005DC00010E0401165F000E175B185B195BDCD76C
:0405EC00006A12008F
:1005F0000401186B050E185D0AE218511625E16E0C
:10060000000E1721E26E200EE66E182BF3D718515C
:100610001625E16E000E1721E26EE66A18071851E2
:100620001625196F000E17211A6F0A0E046E000EA0
:10063000056E14C400F015C401F0C3DD08C000F05D
:1006400009C001F0300E002619C4E1FF1AC4E2FF10
:1006500000C0E6FF0A0E046E000E056E14C400F022
:1006600015C401F0AEDD00C014F401C015F4000E95
:10067000011802E1000E001801E102D01807CFD7DF
:02068000120066
:1006820004011451390806E3300E145D03E3010E30
:08069200006E01D0006A1200A5
:08069A000B6A0B86FF0E120033
:1006A2000C6A0E6A0250D8A46AEF03F001C002F08D
:1006B20000C001F0006A0E860250D8A46AEF03F06F
:1006C20001C002F0016A0E960E880250D8B47CEF87
:1006D20003F00E50035ED8A4D8A081EF03F0D890A7
:1006E20002BE86EF03F0003601360236032E71EFAA
:1006F20003F081EF03F0010E0C6EB6DE89EF03F01A
:10070200020E0C6EA4DE89EF03F0040E0C6E9BDE6B
:020712001200D3
:100714003C0ECF6EB00ECE6E0AC425F30BC426F386
:0E0724000301276B286BCD809E909D801200F4
:1007320004010D6B0AC4E9FF0BC4EAFFEECF0CF40F
:100742000C51000A0EE00CC41CF405DD04010D2B53
:100752000D510A25E96E000E0B21EA6EEECF0CF464
:04076200EFD71200BB
:100766000AC4E9FF0BC4EAFFEECF0CF4000E040145
:100776000D6F000E0D6F000E0D1902E1200E0C1903
:1007860007E0000E0D1902E1090E0C1901E003D075
:100796000A4B0B2BE5D70E6B0F6B106B116B000E14
:1007A6000D1902E12D0E0C1905E1104B112B0A4B08
:1007B6000B2B08D0000E0D1902E12B0E0C1902E1CD
:1007C6000A4B0B2B0AC4E9FF0BC4EAFFEECF0CF46D
:1007D600000E0D6F000E0D6F0CC414F44FDF0052A7
:1007E60018E00EC400F00FC401F00A0E046E000EED
:1007F600056EBDDD300E0C5D026E000E0D59036EEA
:10080600025000240E6F035001200F6F0A4B0B2B72
:10081600D9D71051111108E00E510008006E0FC40F
:1008260001F0000E015604D00EC400F00FC401F012
:020836001200AE
:100838000AC402F00BC403F002C000F003C001F0C8
:10084800024A032A00C0E9FF01C0EAFFEE5201E0B4
:10085800F3D704010A51025C006E0B510358016E74
:0A086800010E005E000E015A12009E
:1008720074DED00E0401146FFEDD0AC414F4FBDD35
:0A0882000BC414F4F8DDDDDD1200F4
:10088C0067DED00E0401146FF1DD0401146BEEDD94
:10089C003FDDD10E0401146FE9DD010E0401146F6C
:1008AC00D3DC00C011F3010E0401146FCDDC00C0C9
:1008BC0013F3010E0401146FC7DC00C0FFF2010E2C
:1008CC000401146FC1DC070E00140201E76F010E66
:1008DC000401146FB9DC00C0E6F2010E0401146FC0
:1008EC00B3DC1F0E00140301186F0401146BACDC95
:1008FC0000C0E5F218C314F492DC00C0FEF211C380
:0C090C0014F48DDC00C0D3F297DD120063
:100918000AC400F00032009E0032009E0032009EA1
:100928000032009E0BC4E1FF0CC4E2FF300E00242D
:10093800E66E010E04010B25E16E000E0C21E26E3D
:100948000F0E0A15006E300E002600C0E6FF020EDC
:0E0958000B25E16E000E0C21E26EE66A120025
:100966000D0E04011C6FACEC00F00A0E04011C6FA6
:06097600ACEC00F01200E1
:0A097C00050E0D6E0D2EFED71200C1
:100986000301296B2A6B000E2A5D02E17F0E295DA9
:1009960012E22B0E2925E16E030E2A21E26EE66A8B
:1009A600010E2925006E000E2A21016E00C029F3D2
:1009B60001C02AF3E8D7226B236B296B2A6B246BC1
:1009C600AB981E6B1F6BAB88F28CAECF24F39D8A5F
:0609D600206B216B1200F2
:1009DC00A69C0BC4AAFF0AC4A9FFA69EA680A8CFFA
:0409EC0000F0120005
:1009F0000401106B116B0AC412F40BC413F4800EC3
:100A00000B19006E800E005C02E1000E0A5D0BE225
:100A1000010E106F000E116F0A510008126F0BC407
:100A200013F4000E135712C414F413C415F40CC4B9
:100A300016F40DC417F4DCDD060E0E6F000E0F6FFA
:100A4000000E006E0F51005C02E10E51000819E229
:100A50000E510C25E16E0F510D21E26E010E0E5D5F
:100A6000006E000E0F59016E00500C25E96E01500A
:100A70000D21EA6EEECFE6FF010E0E5F000E0F5B5A
:100A8000DFD70CC4E1FF0DC4E2FF200EE66E10516B
:100A900011111AE00E6B0F6B0E510C25E96E0F5100
:100AA0000D21EA6EEE50200A03E10E4B0F2BF4D716
:100AB000010E0E5F000E0F5B0E510C25E16E0F5103
:0A0AC0000D21E26E2D0EE66E12000D
:100ACA000AC4F6FF0BC4F7FF0CC4F8FF0900F5CF00
:100ADA0000F0005212E00AC4F6FF0BC4F7FF0CC480
:100AEA00F8FF0900F5CF1CF4ACEC00F0010E04018C
:100AFA000A27000E0B230C23E3D71A0E0D6E0D2EB8
:060B0A00FED700001200FE
:100B10000B820BAE92EF05F0036802680168006873
:080B20000A360232FF0E12003A
:100B280004010A6B0B6B800E0B19006E800E005CC3
:100B380002E1080E0A5D11E20A51010F146F156BEC
:100B4800166B176B186B3ADC6A0E0D6E0D2EFED7FE
:0C0B5800000004010A4B0B2BE6D7120032
:100B640004010B6B0A5109081BE20A0E046E0AC445
:100B740000F0E3DC00C00BF400C00BF40B370B9166
:100B84000B370B910B370B910B370B910A0E046E3D
:100B94000AC400F0D2DC08C000F000500B1302D0ED
:0A0BA4000AC40BF40BC400F01200A9
:100BAE000B6A0A6A096A086A0E6A03340836045028
:100BBE00085E0550D8A0053C095E0650D8A0063C3C
:100BCE000A5E0750D8A0073C0B5EE86AD8A0010E5B
:100BDE000E5E0336070E0C6E0334083609360A36DF
:100BEE000B360E36045003A012D0085E0550D8A066
:100BFE00053C095E0650D8A0063C0A5E0750D8A0F8
:100C0E00073C0B5EE86AD8A0010E0E5E11D00826D6
:100C1E000550D8B0053C09260650D8B0063C0A2629
:100C2E000750D8B0073C0B26E86AD8B0010E0E2646
:100C3E0003360C2ED1D70234083609360A360B3657
:100C4E000E36045003A012D0085E0550D8A0053C05
:100C5E00095E0650D8A0063C0A5E0750D8A0073C95
:100C6E000B5EE86AD8A0010E0E5E11D00826055064
:100C7E00D8B0053C09260650D8B0063C0A260750C7
:100C8E00D8B0073C0B26E86AD8B0010E0E26023605
:100C9E00070E0C6E0234083609360A360B360E363F
:100CAE00045002A012D0085E0550D8A0053C095E83
:100CBE000650D8A0063C0A5E0750D8A0073C0B5E33
:100CCE00E86AD8A0010E0E5E11D008260550D8B0E5
:100CDE00053C09260650D8B0063C0A260750D8B067
:100CEE00073C0B26E86AD8B0010E0E2602360C2EF3
:100CFE00D1D70134083609360A360B360E36045073
:100D0E0002A012D0085E0550D8A0053C095E065020
:100D1E00D8A0063C0A5E0750D8A0073C0B5EE86AD6
:100D2E00D8A0010E0E5E11D008260550D8B0053C95
:100D3E0009260650D8B0063C0A260750D8B0073C04
:100D4E000B26E86AD8B0010E0E260136070E0C6E81
:100D5E000134083609360A360B360E36045001A019
:100D6E0012D0085E0550D8A0053C095E0650D8A0EA
:100D7E00063C0A5E0750D8A0073C0B5EE86AD8A076
:100D8E00010E0E5E11D008260550D8B0053C09267E
:100D9E000650D8B0063C0A260750D8B0073C0B26A2
:100DAE00E86AD8B0010E0E2601360C2ED1D70034CB
:100DBE00083609360A360B360E36045001A012D00C
:100DCE00085E0550D8A0053C095E0650D8A0063C2A
:100DDE000A5E0750D8A0073C0B5EE86AD8A0010E49
:100DEE000E5E11D008260550D8B0053C09260650D7
:100DFE00D8B0063C0A260750D8B0073C0B26E86A46
:100E0E00D8B0010E0E260036070E0C6E00340836D2
:100E1E0009360A360B360E36045000A012D0085E84
:100E2E000550D8A0053C095E0650D8A0063C0A5EC7
:100E3E000750D8A0073C0B5EE86AD8A0010E0E5EE4
:100E4E0011D008260550D8B0053C09260650D8B05A
:100E5E00063C0A260750D8B0073C0B26E86AD8B0E5
:100E6E00010E0E2600360C2ED1D700B00ED0045037
:100E7E0008260550D8B0053C09260650D8B0063CC9
:0C0E8E000A260750D8B0073C0B261200C3
:100E9A00020E0C6E080E0D6E0D2EFED70C2EFCD710
:040EAA000000120032
:100EAE000B0E0C6E570E0D6E0D2EFED70C2EFCD7A4
:060EBE000000000012001C
:100EC400020E0C6E9D0E0D6E0D2EFED70C2EFCD751
:060ED40000000000120006
:100EDA0004010C6B0D6B0AC403F00BC404F00AC4C2
:100EEA0005F00BC406F003C0E9FF04C0EAFFEE50A8
:100EFA00200A04E10C510D1101E110D0010E0C6F12
:100F0A00000E0D6F03C0E9FF04C0EAFF05C0E1FF50
:100F1A0006C0E2FFEECFE6FF054A062A03C001F04B
:100F2A0004C002F0034A042A01C0E9FF02C0EAFF32
:100F3A00EE50000AD8E10AC400F00BC401F0120016
:100F4A000301FD6BFE6B000EFE5D02E10A0EFD5D04
:100F5A000FE2FD5104010525E16E0301FE51040172
:100F6A000621E26E200EE66E0301FD4BFE2BEBD747
:100F7A00FD5104010525E16E0301FE51040106211C
:100F8A00E26EE66A010E0301FD5F000EFE5BFD5193
:100F9A00040105250301FF6FFE5104010621006FBC
:100FAA000A0E046E000E056E066E076E01C400F08E
:100FBA0002C401F003C402F004C403F0F3DD08C064
:100FCA0000F009C001F00AC002F00BC003F0300EB5
:100FDA000026FFC3E1FF00C4E2FF00C0E6FF0A0EDD
:100FEA00046E000E056E066E076E01C400F002C4A0
:100FFA0001F003C402F004C403F0D4DD00C001F41C
:10100A0001C002F402C003F403C004F4000E046E2B
:10101A00031808E10450021805E10450011802E11E
:10102A000050000A01E106D0010E0301FD5F000E27
:06103A00FE5BADD71200C1
:101040000900F5CFE6FF0006FBE10106F9E1120019
:10105000090E0B6E1E0E0C6EE40E0D6E0D2EFED7DD
:0C1060000C2EFCD70B2EFAD7000012005B
:10106C00806A0F01386B2F0E926E92969298899827
:10107C00546BFF0E816E396B870E936EFF0E616E93
:10108C00F19E9382948A8A949386826A3A6B948EA8
:10109C00949C8280949A8B9A9492949094948B8240
:0810AC008B948B90606A120026
:0E10B400300EB16EB36AB26AA192A092120021
:1010C2000401056B066B036B046BFDC3E9FFFEC3F2
:1010D200EAFFEE500008D8B0ECD1FDC3E9FFFEC331
:1010E200EAFF300EEE5C006F016B026B800E02199C
:1010F200006E800E005C02E1080E015DD8B0CED118
:1011020075D1FDC3E9FFFEC3EAFFEE502D0A1AE1D5
:101112000301FF51010A16E1040101510325006E8A
:1011220002510421016EED0E0024E16E010E012038
:10113200E26E630E0125E96E010E0221EA6EEECF28
:10114200E6FF26D0040101510325006E025104215D
:10115200016EED0E0024E16E010E0120E26E030E1F
:10116200026E00C400F0000E016E025005E000366F
:1011720000900136FF0FFAD7780E0026000E0122EA
:1011820001510024E96E02510120EA6EEECFE6FF22
:1011920049D101510325006E02510421016EED0E69
:1011A2000024E16E010E0120E26E030E026E00C405
:1011B20000F0000E016E025005E00036009001368C
:1011C200FF0FFAD7780E0026000E012201510024EB
:1011D200E96E02510120EA6EEECFE6FF0301FF51F4
:1011E200000A27E1010E0201D315016E0150000A27
:1011F20020E1040101510325006E02510421016E18
:10120200ED0E0024026E010E0120036EC80E0125B0
:10121200D96E000E0221DA6E02C0E9FF03C0EAFFB6
:10122200DE50EE10006E02C0E1FF03C0E2FF00C01C
:10123200E6FF0301FF51010A20E1040101510325E8
:10124200006E02510421016EED0E0024026E010EA9
:101252000120036E5B0E0125D96E010E0221DA6EAA
:1012620002C0E9FF03C0EAFFDE50EE10006E02C0CA
:10127200E1FF03C0E2FF00C0E6FFD4D00401015148
:101282000325006E02510421016EED0E0024E16E71
:10129200010E0120E26E030E026E00C400F0000E89
:1012A200016E025005E0003600900136FF0FFAD7BA
:1012B2000401280E0026000E012201510024E96ECD
:1012C20002510120EA6EEECFE6FF0301FF51000A50
:1012D20027E1010E0201D315016E0150000A20E13F
:1012E200040101510325006E02510421016EED0E2D
:1012F2000024026E010E0120036E200E0125D96E1C
:10130200000E0221DA6E02C0E9FF03C0EAFFDE50DE
:10131200EE10006E02C0E1FF03C0E2FF00C0E6FF74
:101322000301FF51010A20E1040101510325006E6E
:1013320002510421016EED0E0024026E010E012005
:10134200036E020E0125D96E010E0221DA6E02C071
:10135200E9FF03C0EAFFDE50EE10006E02C0E1FFBB
:1013620003C0E2FF00C0E6FF5DD004010151032586
:10137200006E02510421016EED0E0024E16E010E99
:101382000120E26E030E026E00C400F0000E016E38
:10139200025005E0003600900136FF0FFAD7040133
:1013A200280E0026000E012201510024E96E02518E
:1013B2000120EA6EEECFE6FF0301FF51010A15E1BB
:1013C200040101510325006E02510421016EED0E4C
:1013D2000024E16E010E0120E26EFA0E0125E96E93
:1013E200000E0221EA6EEECFE6FF1CD00401000ED1
:1013F200061902E1000E0519D8B483D6000E0619AB
:1014020002E1010E0519D8B4C4D6000E061902E194
:10141200020E0519D8B432D7000E061902E1030EE6
:101422000519A3E004010151010F146F180E0125E3
:10143200006E000E0221016EED0E0024E96E010E17
:101442000120EA6EEECF15F4100E0125006E000E9B
:101452000221016EED0E0024E96E010E0120EA6EFA
:10146200EECF16F4080E0125006E000E0221016E69
:10147200ED0E0024E96E010E0120EA6EEECF17F4A4
:10148200ED0E0125E96E010E0221EA6EEECF18F48F
:10149200E2EC01F00401014B022B28D6080E0327CF
:1014A200000E04230301FD4BFE2B0401054B062B0A
:0414B2000CD6120042
:1014B60000C008F00150006E016A026A036A0B6AF6
:1014C6000C6A016A026A036A960E036E0A6A00AE25
:1014D60073EF0AF0081E001E082AD8B4002A0A8EE6
:1014E60000C001F008C000F0086A026A51EC03F07F
:0214F6001200E2
:1014F800020E0301FD6F000EFE6FB3EC04F0040151
:10150800036B046B9D9A2B0E03012925E16E030ED4
:101518002A21E26EE66A000E2A5D02E1160E295DB6
:10152800D8B003D1000E006E2A51005C02E12951A7
:101538001308D8B0FAD0020E0401016F000E026F32
:1015480003012A510401025D04E103012951040148
:10155800015D48E22B0E0125E96E030E0221EA6EB9
:10156800EE503B0A3BE12B0E0125E16E030E0221F2
:10157800E26EE66AD40E03250301FF6F020E040132
:101588000421006F2B0E0301FD2504010A6F030ED1
:101598000301FE2104010B6FB3EC03F0FFC3E1FF6D
:1015A80000C4E2FF00C0E6FF2B0E0301FD25040185
:1015B8000A6F030E0301FE2104010B6F99EC03F07F
:1015C800B3EC04F00401034B042B010E01250301C5
:1015D800FD6F000E040102210301FE6F0401014B9F
:1015E800022BAED7D40E03250301FF6F020E0401B0
:1015F8000421006F2B0E0301FD2504010A6F030E61
:101608000301FE2104010B6FB3EC03F0FFC3E1FFFC
:1016180000C4E2FF00C0E6FFD4C2E6F21F0E0201DA
:10162800D515006E00C018F3D6C2E5F2D7C2FFF296
:10163800D8C213F3070ED915E76F00C014F415ECE0
:1016480001F000C0FEF2070E0201D915016E01C0BB
:10165800E7F2015007080AE2E76B6C0E04010A6F13
:10166800590E0B6F000E0C6F65EC05F018C314F4DF
:1016780015EC01F000C0FEF200500C0802E2020175
:10168800FE6B04010A6B0B6B39EC04F013C30AF40C
:10169800B2EC05F000C00BF4010E0A6F39EC04F04F
:1016A800FFC20AF4B2EC05F000C00BF4020E0A6F98
:1016B80039EC04F0E7C20AF4B2EC05F000C00BF410
:1016C800030E0A6F39EC04F0E6C20AF4B2EC05F036
:1016D80000C00BF4040E0A6F39EC04F018C30AF4C6
:1016E800B2EC05F000C00BF4050E0A6F39EC04F0FB
:1016F800E5C20AF4B2EC05F000C00BF4060E0A6F5E
:1017080039EC04F0070E04010A6F100E0B6F39EC68
:1017180004F00E0E04010A6F5A0E0B6F000E0C6FC8
:1017280065EC05F0B3EC04F012D0D30E04010A6F97
:10173800560E0B6F000E0C6F65EC05F0990E040148
:101748000A6F560E0B6F000E0C6F65EC05F0120059
:101758000450000A12E10550000A0FE10650000A81
:101768000CE10750000A09E1FF0E006EFF0E016E42
:101778007F0E026EFF0E036EA8D0086A096A075032
:10178800D8B457EF0CF00350D8B45CEF0CF002500B
:1017980006180A6E028E068E0E6A02C008F001C094
:1017A8000CF000C00DF004500D5E0550D8A0053CAB
:1017B8000C5E0650D8A0063C085E086A0C6A0D6AE2
:1017C800D8A0EEEF0BF0D890023201320032083286
:1017D800010E0E6E0750035ED8A0FBEF0BF07E0ED5
:1017E8000E240326D8B061EF0CF001EF0CF07E0E4A
:1017F8000E240326D8A066EF0CF0180E0B6E0D36DB
:101808000C3608360036013602360E360450005EB5
:101818000550D8A0053C015E0650D8A0063C025EE3
:1018280006340E120EA01CEF0CF00D8027EF0CF002
:10183800045000260550D8B0053C01260650D8B003
:10184800062802260D900B2E03EF0CF04DEF0CF03E
:10185800D8900036013602360E360450005E055028
:10186800D8A0053C015E0650D8A0063C025E0634AE
:101878000E10010B0D26D8B00C2AD8B4082AD8A40B
:101888004DEF0CF008320C320D32032AD8B461EF58
:101898000CF00AAE089E0850026E0C50016E0D50F6
:1018A800006E69EF0CF0010E4DEC03F069EF0CF0DF
:1018B800020E35EC02F069EF0CF0040E88EC05F02E
:0C18C80069EF0CF0080E28EC02F0120092
:1018D4008B9A070E0C6E3A0E0D6E0D2EFED70C2E43
:1018E400FCD70000B180016A026A800E0218006E03
:1018F400800E050A005C02E1A00E015C13E28B8AF3
:10190400000000000000000000008B9A00000000AE
:101914000000000000000000000000000000014A78
:10192400022AE3D7B1908B9A070E0C6E3A0E0D6E15
:0E1934000D2EFED70C2EFCD700008B8A120061
:10194200580E0201FA6F010EFB6F1C0EFC6F040EA3
:10195200FD6FFF0EF06FFF0EF16F000EF26F000EC3
:10196200F36FFF0EEC6FFF0EED6F000EEE6F000EC9
:10197200EF6FFF0EF66FFF0EF76F000EF86F000E9F
:10198200F96FAC8A900EAB6E948E949C9EAA03D093
:08199200AECF00F0FBD71200FC
:10199A000301FD6BFE6B040101510301FD250401E6
:1019AA000A6F02510301FE2104010B6FEEEC04F0F1
:1019BA0000C0FFF30050000A01E126D0800E030A9E
:1019CA00006E800E0301FE19005C02E1FD51FF0862
:1019DA0001E21AD0FD5104010325E16E0301FE5113
:1019EA0004010421E26EFFC3E6FF680E0C6EE40EEA
:1019FA000D6E0D2EFED70C2EFCD700000301FD4BF9
:101A0A00FE2BFF51000AC7E10301FD510401032522
:101A1A00E16E0301FE5104010421E26EE66A12003E
:101A2A00FFC301F0010E006E015004E00036009081
:101A3A00FF0FFBD700C001F4001EFDC3E9FFFEC380
:101A4A00EAFF0050EF16120EE9260050EF1657EC87
:101A5A0007F004010151EF12120EE95E62EC07F081
:101A6A000151EF14006F0051000A000ED8A4010EB4
:0C1A7A00006F57EC07F000C400F01200F1
:101A8600AEEC02F0D00E0401146F3CEC02F0110E25
:101A96000401146F3CEC02F08EEC01F0D10E04014F
:101AA600146F3CEC02F0010E0401146F2AEC01F0F5
:101AB60000C007F40401146B2AEC01F000C008F41E
:101AC60022EC02F0200E0401096F07AF0AD02D0E9A
:101AD600096FFF0E071B085302E1072B01D008818F
:101AE60007D00751630804E2640E075F310E096FE1
:101AF60009C4FEF3300E096F0751090804E2092BE9
:101B06000A0E075FF9D709C4FFF3300E0725006FE9
:101B16002E0E016F300E076F300E096F085310E05E
:101B260008BD03D0350E076F0BD0320E076F350E8A
:101B3600096F08A101D0087F08AF02D0370E076FE2
:101B460007C402F409C403F40301FD51000A04E1C9
:101B5600B00E0401046F03D00401DF0E046F430EC0
:0E1B6600056F066BFE0E006E030E016E120080
:101B74008B8A000000000000000000008B9A000027
:101B84000000000000000000000000000000000051
:021B940012003D
:101B96000101EB6BEC6B000EEC5D02E1600EEB5DA0
:101BA6000AE2ED0EEB25E16E010EEC21E26EE66A2D
:101BB600EB4BEC2BF0D7FDC30AF4FEC30BF41CEC85
:101BC60004F002014F6B506BFDC3E9FFFEC3EAFF51
:101BD600EE500008D8B08BD0FDC3E9FFFEC3EAFF84
:101BE600200EEE5C0401016F030E006E000E026F04
:101BF600005005E0013701910237FF0FFAD70101C6
:101C0600EB6BEC6B000EEC5D02E1080EEB5D66E241
:101C1600EB5102014F25006E0101EC5102015021EA
:101C2600016EED0E0024E16E010E0120E26E01014F
:101C3600EB5104010125006E0101EC510401022162
:101C4600016E640E0024F66E490E0120F76E000E3A
:101C5600F86E000EF8220900F5CF00F000C0E6FF8E
:101C66000101EB51010F0401146F180E0101EB2560
:101C7600006E000EEC21016EED0E0024E96E010EE1
:101C86000120EA6EEECF15F4100EEB25006E000E65
:101C9600EC21016EED0E0024E96E010E0120EA6EC4
:101CA600EECF16F4080EEB25006E000EEC21016E49
:101CB600ED0E0024E96E010E0120EA6EEECF17F458
:101CC600ED0EEB25E96E010EEC21EA6EEECF18F46F
:101CD600E2EC01F00101EB4BEC2B94D7080E02016C
:101CE6004F27000E50230301FD4BFE2B6DD712002C
:101CF600520E0B6E2B0E0C6E000E0D6E0D2EFED7B9
:0C1D06000C2EFCD70B2EFAD700001200A8
:101D12008B8A0000000000000000000000000000AC
:101D2200000000008B9A000000000000000000008C
:021D320012009D
:101D3400800E0301FE6FFE51000815E2FE51FD15F1
:101D4400016E0150000806E22A0E04011C6FACEC7F
:101D540000F005D0200E04011C6FACEC00F0030170
:081D6400FE33FE9FE8D71200D8
:101D6C00C3EC04F0FDC30AF4FEC30BF48AEC03F0DD
:101D7C008F0E04010A6F590E0B6F000E0C6F65EC81
:101D8C0005F0FDC30AF4FEC30BF4AB0E04010C6F9B
:101D9C00030E0D6FF8EC04F0AB0E0A6F030E0B6F15
:101DAC006DEC07F0AB0E0A6F030E0B6F99EC03F0A2
:101DBC00E40E0A6F5B0E0B6F000E0C6F65EC05F0FA
:101DCC00000E03011F1902E1000E1E1907E1000E9F
:101DDC00281902E1000E271901E1F2D7276B286BB5
:0A1DEC001E6B1F6BB3EC04F0120035
:101DF600310ECD6ECD823C0ECF6EB00ECE6E9E9065
:101E06009F800301256B266B276B286BCD909D90D9
:021E16001200B8
:101E18000F0E0401146F156B166B176B186BE2EC41
:101E280001F0090E0401146F156B166B176B186B14
:101E3800E2EC01F00A0E0401146F010E156F010E99
:101E4800166F010E176F010E186FE2EC01F00B0E02
:101E58000401146F070E156F070E166F070E176F24
:101E6800070E186FE2EC01F00C0E0401146F010E5E
:101E7800156F010E166F010E176F010E186FE2EC49
:101E880001F02A0E0C6E8D0E0D6E0D2EFED70C2E47
:101E9800FCD7000000000301FD6BFE6B800EFE19ED
:101EA800006E800E005C02E1080EFD5D0EE2FD5141
:101EB800010F0401146F156B166B176B186BE2ECAE
:101EC80001F00301FD4BFE2BE9D794EC05F0D00E91
:101ED8000C6EC90E0D6E0D2EFED70C2EFCD7000011
:041EE80000001200E4
:101EEC00FFC301F0010E006E015004E000360090BB
:101EFC00FF0FFBD700C003F4001C0401026F016B41
:101F0C00FDC3E9FFFEC3EAFF006B0051070824E3A1
:101F1C000251EF16120EE9260251EF16BEEC04F038
:101F2C000351EF12BEEC04F0120EE95E0351EF14F4
:101F3C00006E0CE000C401F0010E006E015004E0D4
:101F4C0000360090FF0FFBD7005001134DEC07F04B
:0E1F5C004DEC07F0002BD9D701C400F01200A5
:101F6A00FDC300F00032009E0032009E0032009E47
:101F7A000032009E840E0024F66E5B0EF76E000E91
:101F8A00F722000EF86E000EF8220900F5CF00F0D5
:101F9A00FEC3E1FFFFC3E2FF00C0E6FF010E03013B
:101FAA00FE25E16E000EFF21E26E0F0EFD15006E9A
:101FBA00840E0024F66E5B0EF76E000EF722000EFA
:101FCA00F86E000EF8220900F5CF00F000C0E6FF17
:101FDA00020EFE25E16E000EFF21E26EE66A120095
:101FEA00060E0C6E300E0D6E0D2EFED70C2EFCD783
:041FFA0000001200D1
:101FFE0003C401F0010E006E015004E000360090A3
:10200E00FF0FFBD700C0FFF3001E00C0FEF301C49C
:10201E00E9FF02C4EAFF0050EF16120EE926030193
:10202E00FD6BFD51070816E3FDC300F004C401F07B
:10203E00005004E00132019EFF0FFBD7FE51EF1658
:10204E0001A002D0FF51EF1262EC07F0FF51EF1228
:10205E00FD2BE7D7120EE95E4DEC07F04DEC07F0C5
:02206E0012005E
:102070000401006B0301FEAF0BD0010E0401006FE1
:102080002D0E0301AB6FFD1FFE1FFD4BFE2B05D078
:102090000401006B200E0301AB6FFDC300F0FEC313
:1020A00001F001320032019E01320032019E013204
:1020B0000032019E01320032019E00C0FFF30A0E81
:1020C000046E9FEC02F00A0E046E9FEC02F008C052
:1020D00000F0300E0024AC6FAC51300A02E1200E4B
:1020E000AC6F0A0E046EFFC300F09FEC02F008C054
:1020F00000F0300E0024AD6FFDC301F4FEC302F406
:102100000F0EFD15006EFEC301F0000E011600C09B
:1021100001F401C002F4710E046E020E056EBAECF9
:1021200001F000C003F401C004F403C401F404C4CA
:1021300002F42E0EAE6FE80E046E030E056E03C49D
:1021400000F004C401F0E1EC00F0300E0024AF6FA9
:10215000640E046E000E056E03C400F004C401F0AA
:10216000E1EC00F00A0E046E000E056EE1EC00F0EA
:1021700008C000F009C001F0300E0024B06FB16B50
:10218000B26BB36BAC0E04010A6F030E0B6F6DECF8
:1021900007F00051010A17E1FFC300F0000E016EC5
:1021A000E80E046E030E056EBAEC01F00151002436
:1021B00001016C6F04010251012001016D6F000EDD
:1021C0006E6F6F6F1AD0FFC300F0000E016EE80E45
:1021D000046E030E056EBAEC01F0040101510026F5
:1021E000025101220050000801016C6F01C06DF125
:0C21F000000E6D57000E6E6F6F6F120036
:1021FC0046EC04F0FFC20AF4520E0B6F010E0C6F8A
:10220C008CEC04F03A0E0101546F13C30AF4550E12
:10221C0004010B6F010E0C6F8CEC04F03A0E0101F3
:10222C00576F11C30AF4580E04010B6F010E0C6F9B
:10223C008CEC04F001015A6BE6C20AF40A0E04019C
:10224C000B6F010E0C6F8CEC04F02D0E01010C6F5A
:10225C0018C30AF40D0E04010B6F010E0C6F8CECFD
:10226C0004F02D0E01010F6FE5C20AF4100E0401EB
:10227C000B6F010E0C6F8CEC04F00101126B18C388
:10228C0014F415EC01F000C0FEF211C314F415ECBB
:10229C0001F000C0D3F2FFC214F415EC01F000C041
:1022AC0012F313C314F415EC01F000C000F3030196
:1022BC00FD51010A1EE10A0E04010A6F010E0B6F9B
:1022CC0099EC03F0F40E0A6F5C0E0B6F000E0C6FA2
:1022DC0065EC05F0520E04010A6F010E0B6F99ECC0
:1022EC0003F0F40E0A6F5C0E0B6F000E0C6F65ECB6
:0422FC0005F01200D7
:10230000A6A202D00000FCD7A69CFEC3AAFFFDC374
:10231000A9FFFFC3A8FFA69EA684F2CF00F0F29EFD
:10232000550EA76EAA0EA76EA68200BE02D0F29E20
:1023300001D0F28EA694A1B802D00000FCD7A198DB
:02234000120089
:1023420003C4F6FF04C4F7FF05C4F8FF0900F5CF84
:1023520000F0005218E003C4F6FF04C4F7FF05C4FE
:10236200F8FF0900F5CF00F001C4E1FF02C4E2FF6B
:1023720000C0E6FF0401014B022B010E0327000EF1
:1023820004230523DDD701C4E1FF02C4E2FFE66AAC
:02239200120037
:10239400F80E0201DD6F010EDE6F000EDF6F000E1E
:1023A400E06F5C0EE86F050EE96F000EEA6F000E39
:1023B400EB6F1C0E0301056F030E066F000E076F13
:1023C400000E086F540E016F020E026F140E036F9D
:1023D400040E046F780E0D6F040E0E6F140E0F6F43
:1023E400040E106F440E096F040E0A6F000E0B6F7B
:1023F400000E0C6F949894968B988B969488948680
:0A240400C79EC79C380EC66E12007A
:10240E007DEC2EF09B6A700ED36E9B8CD26A36ECEE
:10241E0008F0546B8B9A8B826AEC0CF0520E0B6E9A
:10242E002B0E0C6E000E0D6E0D2EFED70C2EFCD745
:10243E000B2EFAD70000640E02014D6F000E4E6F88
:10244E0089980101EB6BEC6B000EEC5D02E1800EE6
:10245E00EB5D0AE2530EEB25E16E020EEC21E26E0D
:10246E00E66AEB4BEC2BF0D7530E0201516F020EC6
:10247E00526FB886B06A8A0EAF6EAC84A1EC0CF0C7
:10248E00090E0B6E1E0E0C6EE40E0D6E0D2EFED78B
:10249E000C2EFCD70B2EFAD700000C0E04011C6F6D
:1024AE00ACEC00F0090E0B6E1E0E0C6EE40E0D6EF3
:1024BE000D2EFED70C2EFCD70B2EFAD70000B3EC48
:1024CE0004F0050E04010A6F5B0E0B6F000E0C6F0D
:1024DE0065EC05F00101EB6BEC6B000EEC5D02E1BF
:1024EE000A0EEB5D1CE2030E006E000E016EEBC1D8
:1024FE0004F0ECC105F0BAEC01F0D50E0024E96E43
:10250E00000E0120EA6EEECF0AF4EECF0BF4EECF02
:10251E000CF465EC05F00101EB4BEC2BDED7090E4C
:10252E000B6E1E0E0C6EE40E0D6E0D2EFED70C2EC7
:10253E00FCD70B2EFAD70000B3EC04F080A446D0E3
:10254E00490E04010A6F590E0B6F000E0C6F65ECED
:10255E0005F0B10E04010A6F590E0B6F000E0C6FD1
:10256E0065EC05F00101EB6BEC6B000EEC5D02E12E
:10257E00060EEB5D2AE28B8A310E04011C6FACEC69
:10258E0000F0290E0B6E960E0C6E7F0E0D6E0D2E3C
:10259E00FED70C2EFCD70B2EFAD78B9A300E0401D9
:1025AE001C6FACEC00F0290E0B6E960E0C6E7F0EAF
:1025BE000D6E0D2EFED70C2EFCD70B2EFAD7B3ECCC
:1025CE0004F00101EB4BEC2BD0D709D0F50E040132
:1025DE000A6F570E0B6F000E0C6F65EC05F06D0E4B
:1025EE0004010A6F580E0B6F000E0C6F65EC05F0B0
:1025FE00530E0201516F020E526F0401016B026BFA
:10260E0051C203F452C204F4CDEC0CF051C20AF4E0
:10261E0052C20BF499EC03F0020E0B6EA00E0C6E70
:10262E00920E0D6E0D2EFED70C2EFCD70B2EFAD75A
:10263E0000000001D06B530E0201516F020E526F5B
:10264E00700E0401016F000E026F51C203F452C2EC
:10265E0004F4CDEC0CF051C20AF452C20BF499EC16
:10266E0003F0040E02015125E96E000E5221EA6EAE
:10267E00300EEE5C0001D06F0A0ED003F3CFD0F017
:10268E00050E02015125E96E000E5221EA6E300E42
:10269E00EE5C006E00500001D0270F0ED017530EC7
:1026AE000201516F020E526F800E0401016F000E77
:1026BE00026F51C203F452C204F4CDEC0CF0020EC0
:1026CE000B6EA00E0C6E920E0D6E0D2EFED70C2EF6
:1026DE00FCD70B2EFAD7000051C20AF452C20BF4EB
:1026EE0099EC03F0060E02015125E16E000E522107
:1026FE00E26EE66A040E512504010A6F000E020115
:10270E00522104010B6FB3EC03F000C0D3F001C0F3
:10271E00D4F0090E02015125E16E000E5221E26E37
:10272E00E66A070E512504010A6F000E02015221BE
:10273E0004010B6FB3EC03F000C0D1F001C0D2F076
:10274E000001D451015C02E1D351005C0BE2000E9A
:10275E00006ED251005C02E1D151000803E2010E7D
:10276E001F6E01D01F6ACC0E04010A6F5B0E0B6F39
:10277E00000E0C6F65EC05F0300E1F2404011C6F6B
:10278E00ACEC00F0B3EC04F01D6A1E6A530E0201AD
:10279E00516F020E526FA00E0401016F000E026FF8
:1027AE0051C203F452C204F4CDEC0CF051C20AF43F
:1027BE0052C20BF499EC03F0060E02015125E96E9C
:1027CE00000E5221EA6E300EEE5C006E016A000EB3
:1027DE00015A640E046E000E056EBAEC01F000C0D4
:1027EE00FBF301C0FCF3FBC31DF0FCC31EF0070E90
:1027FE005125E96E000E5221EA6E300EEE5C006E2F
:10280E00016A000E015A0A0E046E000E056EBAEC35
:10281E0001F000500301FB251D6E0150FC211E6EC0
:10282E00080E02015125E96E000E5221EA6E300E9D
:10283E00EE5C006E016A000E015A00501D2601501A
:10284E001E22050E5125E96E000E5221EA6EEE5043
:10285E002D0A06E11D5000081D6E1E50000E1E565C
:10286E00800E1E18006E800EFE0A005C02E1D40E71
:10287E001D5C0BE3800E010A006E800E1E18005CBC
:10288E0002E11D502C0801E302D01D6A1E6A1DC014
:10289E0000F01EC001F05BEC0AF0000E046E000E9C
:1028AE00056E480E066E850E076EACEC0BF000C082
:1028BE007DF101C07EF102C07FF103C080F1B3EC67
:1028CE0004F0500E04010A6F5B0E0B6F000E0C6FBE
:1028DE0065EC05F05AEC08F0B180050E0B6E0F0E8C
:1028EE000C6EF10E0D6E0D2EFED70C2EFCD70B2E90
:1028FE00FAD7B190B3CF01F0006ACE500024010197
:10290E00796F000E01207A6F000E7B6F7C6FA1A293
:10291E0008D0000E7927000E7A23010E7B23000EBD
:10292E007C2379C100F07AC101F07BC102F07CC139
:10293E0003F00332023201320032039E00C079F1FD
:10294E0001C07AF102C07BF103C07CF100C001F43A
:10295E0001C002F402C003F403C004F4AB0E040180
:10296E00056F030E066FA5EC07F0AB0E04010A6FA0
:10297E00030E0B6F99EC03F0EF0E0A6F5C0E0B6FEC
:10298E00000E0C6F65EC05F0B3EC04F0180E0401AC
:10299E000A6F5B0E0B6F000E0C6F65EC05F0F29E6E
:1029AE005AEC08F06AEC0CF0B3CF01F0006ACE508E
:1029BE0000240101796F000E01207A6F000E7B6FEB
:1029CE007C6FA1A208D0000E7927000E7A23010E8B
:1029DE007B23000E7C2379C100F07AC101F07BC10C
:1029EE0002F07CC103F00332023201320032039E48
:1029FE0000C079F101C07AF102C07BF103C07CF115
:102A0E0000C001F401C002F402C003F403C004F4D8
:102A1E00AB0E0401056F030E066FA5EC07F0AB0EAF
:102A2E0004010A6F030E0B6F99EC03F0E50E0A6FAB
:102A3E005C0E0B6F000E0C6F65EC05F0B3EC04F042
:102A4E00F28E7D0E04010A6F5A0E0B6F000E0C6F84
:102A5E0065EC05F028EC08F002014F6B506B800E10
:102A6E000301FD6F0F0EFE6FFF6B15EC0DF0F5EC15
:102A7E000FF0800E016F0F0E026F036B330E046F9B
:102A8E00FFEC0FF0F5EC0FF0800EFD6F0F0EFE6FEA
:102A9E00FF6B76EC0FF000C024F3F5EC0FF0940E04
:102AAE000A6F5B0E0B6F000E0C6F65EC05F00301E9
:102ABE00AB6B24C3FDF3AB0EFE6F030EFF6FB5ECD5
:102ACE000FF0AB0E04010A6F030E0B6F99EC03F0BF
:102ADE00A00E0A6F5C0E0B6F000E0C6F65EC05F00E
:102AEE000101EB6BEC6B000EEC5D02E1060EEB5D93
:102AFE002AE2800E0301FD6F0F0EFE6FFF6B76EC68
:102B0E000FF000C024F3F5EC0FF0720E0101EB256F
:102B1E00E16E010EEC21E26E24C3E6FF0301AB6B06
:102B2E0024C3FDF3AB0EFE6F030EFF6FB5EC0FF07B
:102B3E00AB0E04010A6F030E0B6F99EC03F001014B
:102B4E00EB4BEC2BD0D77A0E04010A6F5C0E0B6F99
:102B5E00000E0C6F65EC05F0800E0301FD6F0F0E7D
:102B6E00FE6FFF6B76EC0FF000C024F30301AB6B2E
:102B7E0024C3FDF3AB0EFE6F030EFF6FB5EC0FF02B
:102B8E00AB0E04010A6F030E0B6F99EC03F0B3EC5E
:102B9E0004F03E0E04010A6F5B0E0B6F000E0C6FFD
:102BAE0065EC05F0800E0301FD6F0F0EFE6FFF6BDF
:102BBE0015EC0DF0800E016F0F0E026F036BCC0E35
:102BCE00046FFFEC0FF0800E0401016F0F0E026F09
:102BDE00036B440E046FFFEC0FF0F5EC0FF0800E5C
:102BEE00FD6F0F0EFE6FFF6B15EC0DF0800E016F7B
:102BFE000F0E026F036BCC0E046FFFEC0FF0800E06
:102C0E000401016F0F0E026F036BBE0E046FFFEC1B
:102C1E000FF0800EFD6F0F0EFE6FFF6B76EC0FF058
:102C2E0000C01BF0000E1C6E800E0301FD6F0F0E18
:102C3E00FE6FFF6B76EC0FF000C003F0026A1B50C4
:102C4E000224006E1C500320016E00C019F001C05A
:102C5E001AF000C0FDF301C0FEF338EC10F0AB0E1D
:102C6E0004010A6F030E0B6F6DEC07F0AB0E0A6FCB
:102C7E00030E0B6F1CEC04F000C070F101C071F17B
:102C8E00AB0E0024016F030E0120026FDB0E036FEB
:102C9E005C0E046F000E056FA1EC11F0AB0E04017B
:102CAE000A6F030E0B6F99EC03F0B3EC04F0B3EC68
:102CBE0004F0C80E04010A6F5A0E0B6F000E0C6F53
:102CCE0065EC05F0280EC86ECAEC11F0480E040132
:102CDE000A6F5A0E0B6F000E0C6F65EC05F00E0EA0
:102CEE0004010A6F400E0B6F39EC04F081B242D032
:102CFE002B0E04010A6F5A0E0B6F000E0C6F65EC53
:102D0E0005F004010A6B500E0B6F39EC04F0010E46
:102D1E0004010A6F590E0B6F39EC04F00E0E04010C
:102D2E000A6FB2EC05F000C00BF4020E0A6F39EC1C
:102D3E0004F0030E04010A6F020E0B6F39EC04F05F
:102D4E00040E04010A6F010E0B6F39EC04F0050E30
:102D5E0004010A6F050E0B6F39EC04F0120E04011C
:102D6E000A6FB2EC05F000C00BF4060E0A6F39ECD8
:102D7E0004F009D0620E04010A6F5B0E0B6F000E99
:102D8E000C6F65EC05F0010E0301FD6FFEEC10F00B
:102D9E00B3EC04F0B3EC04F0EF0E04010A6F590E1D
:102DAE000B6F000E0C6F65EC05F00301FD6B43EC31
:102DBE000DF000C00AF401C00BF499EC03F0B3EC73
:102DCE0004F0520E0B6E2B0E0C6E000E0D6E0D2EB1
:102DDE00FED70C2EFCD70B2EFAD70000B3EC04F066
:102DEE001D0E04010A6F580E0B6F000E0C6F65EC72
:102DFE0005F0F18C0101816B826BF292F288B90EB3
:102E0E0004010A6F580E0B6F000E0C6F65EC05F087
:102E1E00D08E9F8A9E8AAB88F28CF28E0101706BE7
:102E2E00716B80A4F0D1260E04010A6F590E0B6F40
:102E3E00000E0C6F65EC05F08B9A030E0C6E120EE5
:102E4E000D6E0D2EFED70C2EFCD7000002014F6B1F
:102E5E00506B0101896B8A6B0101706B716B020102
:102E6E0050510101715D04E102014F510101705D8C
:102E7E00D8B091D157D1BAEC0DF0BAEC0DF0BAEC46
:102E8E000DF0BAEC0DF0BAEC0DF0BAEC0DF0BAECA8
:102E9E000DF0BAEC0DF0BAEC0DF0BAEC0DF0BAEC98
:102EAE000DF0BAEC0DF0BAEC0DF0BAEC0DF0BAEC88
:102EBE000DF089EC0EF0BAEC0DF0BAEC0DF0BAECA8
:102ECE000DF0BAEC0DF0BAEC0DF0BAEC0DF0BAEC68
:102EDE000DF0BAEC0DF051D1BAEC0DF0BAEC0DF0DC
:102EEE00BAEC0DF0BAEC0DF0BAEC0DF0BAEC0DF048
:102EFE00BAEC0DF089EC0EF0BAEC0DF0BAEC0DF068
:102F0E00BAEC0DF0BAEC0DF0BAEC0DF0BAEC0DF027
:102F1E00BAEC0DF0BAEC0DF0BAEC0DF0BAEC0DF017
:102F2E00BAEC0DF0BAEC0DF0BAEC0DF0BAEC0DF007
:102F3E00BAEC0DF0BAEC0DF020D1BAEC0DF0BAEC03
:102F4E000DF0BAEC0DF0BAEC0DF0BAEC0DF0BAECE7
:102F5E000DF0BAEC0DF0BAEC0DF0BAEC0DF0BAECD7
:102F6E000DF0BAEC0DF0BAEC0DF0BAEC0DF0BAECC7
:102F7E000DF0BAEC0DF0BAEC0DF0BAEC0DF0BAECB7
:102F8E000DF0BAEC0DF0BAEC0DF0BAEC0DF0BAECA7
:102F9E000DF0BAEC0DF089EC0EF0EFD0BAEC0DF0AE
:102FAE00BAEC0DF0BAEC0DF0BAEC0DF0BAEC0DF087
:102FBE00BAEC0DF0BAEC0DF0BAEC0DF0BAEC0DF077
:102FCE00BAEC0DF0BAEC0DF0BAEC0DF0BAEC0DF067
:102FDE00BAEC0DF0BAEC0DF0BAEC0DF0BAEC0DF057
:102FEE00BAEC0DF0BAEC0DF0BAEC0DF0BAEC0DF047
:102FFE00BAEC0DF0BAEC0DF089EC0EF0BED0BAECD6
:10300E000DF0BAEC0DF0BAEC0DF0BAEC0DF0BAEC26
:10301E000DF0BAEC0DF0BAEC0DF0BAEC0DF0BAEC16
:10302E000DF0BAEC0DF0BAEC0DF0BAEC0DF0BAEC06
:10303E000DF0BAEC0DF0BAEC0DF0BAEC0DF0BAECF6
:10304E000DF0BAEC0DF0BAEC0DF0BAEC0DF0BAECE6
:10305E000DF0BAEC0DF0BAEC0DF089EC0EF08DD04F
:10306E00BAEC0DF0BAEC0DF0BAEC0DF0BAEC0DF0C6
:10307E00BAEC0DF0BAEC0DF0BAEC0DF0BAEC0DF0B6
:10308E00BAEC0DF0BAEC0DF0BAEC0DF0BAEC0DF0A6
:10309E00BAEC0DF0BAEC0DF0BAEC0DF0BAEC0DF096
:1030AE00BAEC0DF0BAEC0DF0BAEC0DF0BAEC0DF086
:1030BE00BAEC0DF0BAEC0DF0BAEC0DF089EC0EF0A6
:1030CE005CD0BAEC0DF0BAEC0DF0BAEC0DF0BAEC37
:1030DE000DF0BAEC0DF0BAEC0DF0BAEC0DF089EC87
:1030EE000EF0BAEC0DF0BAEC0DF0BAEC0DF0BAEC45
:1030FE000DF0BAEC0DF0BAEC0DF0BAEC0DF089EC67
:10310E000EF0BAEC0DF0BAEC0DF0BAEC0DF0BAEC24
:10311E000DF0BAEC0DF0BAEC0DF0BAEC0DF089EC46
:10312E000EF02BD0000E8A1902E1000E8919D8B4C8
:10313E00A2D6000E8A1902E1010E8919D8B4CCD696
:10314E00000E8A1902E1020E8919D8B4F6D6000EC5
:10315E008A1902E1030E8919D8B420D7000E8A19F4
:10316E0002E1040E8919D8B44AD7000E8A1902E179
:10317E00050E8919D8B474D7A4D70101000E006EBC
:10318E008A51005C02E18951050802E2896B8A6B63
:10319E00704B712B64D6894B8A2B090E0B6E1E0E4B
:1031AE000C6EE40E0D6E0D2EFED70C2EFCD70B2ED4
:1031BE00FAD700006AEC0CF0440E04010A6F5C0EA4
:1031CE000B6F000E0C6F65EC05F04FC214F450C27D
:1031DE0015F4AB0E0401166F030E176FF8EC02F028
:1031EE00AB0E0A6F030E0B6F99EC03F0B3EC04F009
:1031FE0002014F4B502B000E505D02E13C0E4F5D15
:10320E00D8A02AD609D0930E04010A6F580E0B6F60
:10321E00000E0C6F65EC05F03C0E04010A6F570EA4
:10322E000B6F000E0C6F65EC05F0FBEC0EF0140E40
:10323E0004010A6F000E0B6F8AEC03F0240EAD6EC4
:10324E00B3EC04F0000E0301281902E1000E271959
:10325E0001E1F8D7230EAD6EB3EC04F00101706BF3
:10326E00716BC3EC04F05D0E04010A6F560E0B6F0A
:10327E00000E0C6F65EC05F0020E04010A6F590E7C
:10328E000B6F000E0C6F65EC05F081A60AD0B20E26
:10329E0004010A6F5B0E0B6F000E0C6F65EC05F0F0
:1032AE0009D0BF0E04010A6F5B0E0B6F000E0C6F80
:1032BE0065EC05F0000E81B6010E04011C6F300E98
:1032CE001C27ACEC00F0290E04011C6FACEC00F0D6
:1032DE00B3EC04F08B82F10E04010A6F5A0E0B6FE1
:1032EE00000E0C6F65EC05F00CEC0FF0DD0E0A6FA6
:1032FE005A0E0B6F000E0C6F65EC05F094EC05F09A
:10330E00B3EC04F08B8280A4D9D0B3EC04F00101AD
:10331E00EB6BEC6B000EEC5D02E10A0EEB5DD8B0D0
:10332E00C4D06F0E04010A6F570E0B6F000E0C6F98
:10333E0065EC05F0300E0101EB2504011C6FACECC1
:10334E0000F0B3EC04F002014F6B506B000E505DB9
:10335E0002E1080E4F5DD8B09BD0ED0E4F25E16E09
:10336E00010E5021E26EEBC100F0ECC101F000360F
:10337E00009001360036009001360036009001367E
:10338E00780E0026000E01224F510024E96E505196
:10339E000120EA6EC80E4F25D96E000E5021DA6E4E
:1033AE00DE50EE10006E00C0E6FFED0E4F25E96E0A
:1033BE00010E5021EA6EEECFFDF39AEC0EF0F70EF1
:1033CE0004010A6F5C0E0B6F000E0C6F65EC05F0BE
:1033DE008B0E02014F25E16E010E5021E26EEBC104
:1033EE0000F0ECC101F0003600900136003600907E
:1033FE000136003600900136280E0026000E0122FE
:10340E004F510024E96E50510120EA6E200E4F25D7
:10341E00D96E000E5021DA6EDE50EE10006E00C036
:10342E00E6FF8B0E4F25E96E010E5021EA6EEECFB0
:10343E00FDF39AEC0EF002014F51010F0401146FCF
:10344E00156B166B8B0E02014F25E96E010E502186
:10345E00EA6EEECF17F4ED0E4F25E96E010E5021F8
:10346E00EA6EEECF18F4E2EC01F0090E0B6E1E0EB2
:10347E000C6EE40E0D6E0D2EFED70C2EFCD70B2E01
:10348E00FAD70000B3EC04F002014F4B502B5ED77D
:10349E00B3EC04F01E0E0301FD6F000EFE6FB6ECD2
:1034AE000EF00101EB4BEC2B35D7B3EC04F0320EE2
:1034BE000301FD6F000EFE6FB6EC0EF0B3EC04F0E0
:1034CE006AEC0CF07BEC0EF0010E0101836F000E26
:1034DE00846F876B886B856B866BC3EC04F08B9A5D
:1034EE00FD6BFEEC10F011C314F415EC01F000C0EE
:1034FE00D3F213C314F415EC01F000C000F3FFC2B5
:10350E0014F415EC01F000C012F33F0E0201FF158A
:10351E000401146F15EC01F000C012F3AB0E016F35
:10352E00030E026F030E006E000E016EE7C204F072
:10353E00000E056EBAEC01F0130E0024E96E010EBA
:10354E000120EA6EEECF03F4EECF04F4EECF05F4D5
:10355E00A1EC11F0AB0E04010A6F030E0B6F99EC88
:10356E0003F0200E1C6FACEC00F00AC11CF4ACECA6
:10357E0000F00BC11CF4ACEC00F0200E04011C6F2B
:10358E00ACEC00F0AB0E0401016F030E026F030EE4
:10359E00006E000E016EFEC204F0000E056EBAEC57
:1035AE0001F02B0E0024E96E010E0120EA6EEECF23
:1035BE0003F4EECF04F4EECF05F4A1EC11F0AB0E54
:1035CE0004010A6F030E0B6F99EC03F0200E1C6FB3
:1035DE00ACEC00F0320E04011C6FACEC00F0300EBF
:1035EE0004011C6FACEC00F010C11CF4ACEC00F04C
:1035FE0011C11CF4ACEC00F0200E04011C6FACECFD
:10360E0000F02C0E04011C6FACEC00F0520E040105
:10361E000A6F010E0B6F99EC03F02C0E1C6FACECC5
:10362E0000F0CF0E04010A6F5C0E0B6F000E0C6FD4
:10363E0065EC05F03B0E04011C6FACEC00F0800E47
:10364E000301FD6F0F0EFE6FFF6B15EC0DF0800E7C
:10365E00016F0F0E026F036BCC0E046FFFEC0FF0B9
:10366E00800E0401016F0F0E026F036B440E046F88
:10367E00FFEC0FF0F5EC0FF0800EFD6F0F0EFE6FEE
:10368E00FF6B15EC0DF0800E016F0F0E026F036BCA
:10369E00CC0E046FFFEC0FF0800E0401016F0F0EC5
:1036AE00026F036BBE0E046FFFEC0FF0800EFD6F0A
:1036BE000F0EFE6FFF6B76EC0FF000C01BF0000ECE
:1036CE001C6E800E0301FD6F0F0EFE6FFF6B76EC0E
:1036DE000FF000C003F0026A1B500224006E1C5053
:1036EE000320016E00C019F001C01AF000C0FDF3F6
:1036FE0001C0FEF338EC10F0AB0E04010A6F030E9E
:10370E000B6F6DEC07F0AB0E0A6F030E0B6F1CEC1C
:10371E0004F000C070F101C071F1AB0E0024016F16
:10372E00030E0120026FE00E036F5C0E046F000E9D
:10373E00056FA1EC11F0AB0E04010A6F030E0B6FB7
:10374E0099EC03F0B3EC04F001016B6B1F50010A0E
:10375E0032E1000E0001D25D04E1030112510001BD
:10376E00D15D0CE2000E006ED451005C03E1D3512A
:10377E000301125D03E201016B6B03D00101010E27
:10378E006B6F6B51010A0AE10A0E0401146F156B7F
:10379E00166B176B186BE2EC01F00DD00A0E0401DC
:1037AE00146FD0C015F4D0C016F4D0C017F4D0C02A
:1037BE0018F4E2EC01F0530E0301196F020E1A6FAA
:1037CE0083D019C301F41AC302F4730E0401036FFC
:1037DE005B0E046F000E056FA1EC11F0E7C202F054
:1037EE00000E036E023603360290025003011925B5
:1037FE00E96E03501A21EA6EEECFABF3010E1925D6
:10380E00006E000E1A21016E02500024E96E035064
:10381E000120EA6EEECFACF30AC1ADF30BC1AEF3ED
:10382E00AF6BAB0EFD6F030EFE6FCBEC0DF072D0D7
:10383E0019C301F41AC302F4030E006E000E016EDA
:10384E00FEC204F0000E056EBAEC01F02B0E002441
:10385E00E96E010E0120EA6EEECF03F4EECF04F412
:10386E00EECF05F4A1EC11F0040E03011925E16E63
:10387E00000E1A21E26EE66A19C3FDF31AC3FEF3B7
:10388E00CBEC0DF047D052C1ABF353C1ACF355C1E5
:10389E00ADF356C1AEF30301AF6BAB0EFD6F030E6E
:1038AE00FE6FFF6B61EC08F035D0AEC3ADF37F0E4B
:1038BE000301AE6FAF6BAB0EFD6F030EFE6F010E0D
:1038CE00FF6F61EC08F026D0000E0101861902E1AF
:1038DE00000E8519D8B475D7000E861902E1010EB7
:1038EE008519A6E0000E861902E1020E8519CBE0BD
:1038FE00000E861902E1030E8519C5E0000E861929
:10390E0002E1040E8519D1E0000E861902E1050EC2
:10391E008519CBE00101854B862B000E006E86517A
:10392E00005C02E18551050802E2856B866B1F5033
:10393E00010A10E16B51010A0DE10A0E0401146F28
:10394E00156B166B176B186BE2EC01F06AEC0CF052
:10395E00EAEF20F00201D351000A1BE1970E040199
:10396E000A6F5A0E0B6F000E0C6F65EC05F06AECC9
:10397E000CF08B9A050E0B6E0F0E0C6EF10E0D6E7B
:10398E000D2EFED70C2EFCD70B2EFAD703011C6B77
:10399E001D6B0301020E1B5DD8B0AED11C6B1D6BEF
:1039AE000101876B886B57D1BAEC0DF0BAEC0DF0B4
:1039BE00BAEC0DF0BAEC0DF0BAEC0DF0BAEC0DF06D
:1039CE00BAEC0DF0BAEC0DF0BAEC0DF0BAEC0DF05D
:1039DE00BAEC0DF0BAEC0DF0BAEC0DF0BAEC0DF04D
:1039EE0089EC0EF089EC0EF0BAEC0DF0BAEC0DF09D
:1039FE00BAEC0DF0BAEC0DF0BAEC0DF0BAEC0DF02D
:103A0E00BAEC0DF0BAEC0DF052D1BAEC0DF0BAECF6
:103A1E000DF0BAEC0DF0BAEC0DF0BAEC0DF0BAEC0C
:103A2E000DF089EC0EF089EC0EF0BAEC0DF0BAEC5C
:103A3E000DF0BAEC0DF0BAEC0DF0BAEC0DF0BAECEC
:103A4E000DF0BAEC0DF0BAEC0DF0BAEC0DF0BAECDC
:103A5E000DF0BAEC0DF0BAEC0DF0BAEC0DF0BAECCC
:103A6E000DF0BAEC0DF0BAEC0DF021D1BAEC0DF070
:103A7E00BAEC0DF0BAEC0DF0BAEC0DF0BAEC0DF0AC
:103A8E00BAEC0DF0BAEC0DF0BAEC0DF0BAEC0DF09C
:103A9E00BAEC0DF0BAEC0DF0BAEC0DF0BAEC0DF08C
:103AAE00BAEC0DF0BAEC0DF0BAEC0DF0BAEC0DF07C
:103ABE00BAEC0DF0BAEC0DF0BAEC0DF0BAEC0DF06C
:103ACE00BAEC0DF089EC0EF089EC0EF0F0D0BAECF9
:103ADE000DF0BAEC0DF0BAEC0DF0BAEC0DF0BAEC4C
:103AEE000DF0BAEC0DF089EC0EF089EC0EF0BAEC9C
:103AFE000DF0BAEC0DF0BAEC0DF0BAEC0DF0BAEC2C
:103B0E000DF0BAEC0DF089EC0EF089EC0EF0BAEC7B
:103B1E000DF0BAEC0DF0BAEC0DF0BAEC0DF0BAEC0B
:103B2E000DF0BAEC0DF089EC0EF089EC0EF0BFD072
:103B3E00BAEC0DF0BAEC0DF0BAEC0DF0BAEC0DF0EB
:103B4E00BAEC0DF0BAEC0DF0BAEC0DF0BAEC0DF0DB
:103B5E00BAEC0DF0BAEC0DF0BAEC0DF089EC0EF0FB
:103B6E00BAEC0DF0BAEC0DF089EC0EF089EC0EF01B
:103B7E00BAEC0DF0BAEC0DF0BAEC0DF089EC0EF0DB
:103B8E00BAEC0DF0BAEC0DF089EC0EF089EC0EF0FB
:103B9E008ED0BAEC0DF0BAEC0DF0BAEC0DF0BAEC2A
:103BAE000DF0BAEC0DF0BAEC0DF089EC0EF089ECDC
:103BBE000EF0BAEC0DF0BAEC0DF0BAEC0DF0BAEC6A
:103BCE000DF0BAEC0DF0BAEC0DF089EC0EF089ECBC
:103BDE000EF0BAEC0DF0BAEC0DF0BAEC0DF0BAEC4A
:103BEE000DF0BAEC0DF0BAEC0DF0BAEC0DF0BAEC3B
:103BFE000DF05DD0BAEC0DF0BAEC0DF0BAEC0DF0A4
:103C0E00BAEC0DF0BAEC0DF0BAEC0DF0BAEC0DF01A
:103C1E00BAEC0DF0BAEC0DF0BAEC0DF0BAEC0DF00A
:103C2E00BAEC0DF0BAEC0DF0BAEC0DF0BAEC0DF0FA
:103C3E00BAEC0DF0BAEC0DF0BAEC0DF0BAEC0DF0EA
:103C4E00BAEC0DF0BAEC0DF0BAEC0DF0BAEC0DF0DA
:103C5E00BAEC0DF02CD00101000E881902E1000E15
:103C6E008719D8B4A1D6000E881902E1010E871962
:103C7E00D8B4CBD6000E881902E1020E8719D8B43B
:103C8E00F5D6000E881902E1030E8719D8B41FD796
:103C9E00000E881902E1040E8719D8B449D7000E18
:103CAE00881902E1050E8719D8B473D7A3D701017D
:103CBE00800E006E800E8819005C02E187510408A8
:103CCE0002E2876B886B874B882B03011C4B1D2BE5
:103CDE000201D351010F016E026A000E0222800E04
:103CEE0003011D19006E800E0218005C02E10150E6
:103CFE001C5DD8A058D667D21C6B1D6B0A0E046EC5
:103D0E0000C300F09FEC02F008C000F000C0FBF30F
:103D1E001BD2BAEC0DF0BAEC0DF0BAEC0DF0BAEC19
:103D2E000DF0BAEC0DF0BAEC0DF0BAEC0DF0BAECF9
:103D3E000DF0BAEC0DF0BAEC0DF0BAEC0DF0BAECE9
:103D4E000DF0BAEC0DF089EC0EF089EC0EF089EC6A
:103D5E000EF0BAEC0DF0BAEC0DF0BAEC0DF0BAECC8
:103D6E000DF0BAEC0DF0BAEC0DF0BAEC0DF0BAECB9
:103D7E000DF013D2BAEC0DF0BAEC0DF0BAEC0DF06A
:103D8E00BAEC0DF0BAEC0DF089EC0EF089EC0EF0F9
:103D9E0089EC0EF0BAEC0DF0BAEC0DF0BAEC0DF0B9
:103DAE00BAEC0DF0BAEC0DF0BAEC0DF0BAEC0DF079
:103DBE00BAEC0DF0BAEC0DF0BAEC0DF0BAEC0DF069
:103DCE00BAEC0DF0BAEC0DF0BAEC0DF0BAEC0DF059
:103DDE00BAEC0DF0E2D1BAEC0DF0BAEC0DF0BAEC93
:103DEE000DF0BAEC0DF0BAEC0DF0BAEC0DF0BAEC39
:103DFE000DF0BAEC0DF0BAEC0DF0BAEC0DF0BAEC29
:103E0E000DF0BAEC0DF0BAEC0DF0BAEC0DF0BAEC18
:103E1E000DF0BAEC0DF0BAEC0DF0BAEC0DF0BAEC08
:103E2E000DF0BAEC0DF0BAEC0DF089EC0EF089EC59
:103E3E000EF089EC0EF0B1D1BAEC0DF0BAEC0DF03B
:103E4E00BAEC0DF0BAEC0DF0BAEC0DF089EC0EF008
:103E5E00BAEC0DF089EC0EF0BAEC0DF0BAEC0DF0F8
:103E6E00BAEC0DF0BAEC0DF0BAEC0DF089EC0EF0E8
:103E7E00BAEC0DF089EC0EF0BAEC0DF0BAEC0DF0D8
:103E8E00BAEC0DF0BAEC0DF0BAEC0DF089EC0EF0C8
:103E9E00BAEC0DF089EC0EF080D1BAEC0DF0BAEC64
:103EAE000DF0BAEC0DF0BAEC0DF0BAEC0DF0BAEC78
:103EBE000DF0BAEC0DF0BAEC0DF0BAEC0DF0BAEC68
:103ECE000DF0BAEC0DF0BAEC0DF089EC0EF0BAEC88
:103EDE000DF0BAEC0DF089EC0EF0BAEC0DF0BAEC78
:103EEE000DF0BAEC0DF0BAEC0DF089EC0EF0BAEC68
:103EFE000DF0BAEC0DF089EC0EF04FD1BAEC0DF0DE
:103F0E00BAEC0DF0BAEC0DF0BAEC0DF0BAEC0DF017
:103F1E00BAEC0DF089EC0EF089EC0EF0BAEC0DF067
:103F2E00BAEC0DF0BAEC0DF0BAEC0DF0BAEC0DF0F7
:103F3E00BAEC0DF089EC0EF089EC0EF0BAEC0DF047
:103F4E00BAEC0DF0BAEC0DF0BAEC0DF0BAEC0DF0D7
:103F5E00BAEC0DF0BAEC0DF0BAEC0DF01ED1BAECD5
:103F6E000DF0BAEC0DF0BAEC0DF0BAEC0DF0BAECB7
:103F7E000DF0BAEC0DF0BAEC0DF089EC0EF0BAECD7
:103F8E000DF0BAEC0DF0BAEC0DF0BAEC0DF0BAEC97
:103F9E000DF089EC0EF089EC0EF089EC0EF0BAEC17
:103FAE000DF0BAEC0DF0BAEC0DF0BAEC0DF0BAEC77
:103FBE000DF0BAEC0DF0BAEC0DF089EC0EF0EDD080
:103FCE00BAEC0DF0BAEC0DF0BAEC0DF0BAEC0DF057
:103FDE00BAEC0DF089EC0EF089EC0EF089EC0EF0D7
:103FEE00BAEC0DF0BAEC0DF0BAEC0DF0BAEC0DF037
:103FFE00BAEC0DF0BAEC0DF0BAEC0DF0BAEC0DF027
:10400E00BAEC0DF0BAEC0DF0BAEC0DF0BAEC0DF016
:10401E00BAEC0DF0BAEC0DF0BAEC0DF089EC0EF036
:10402E00BCD0BAEC0DF0BAEC0DF0BAEC0DF0BAEC67
:10403E000DF0BAEC0DF0BAEC0DF0BAEC0DF089EC17
:10404E000EF0BAEC0DF0BAEC0DF0BAEC0DF0BAECD5
:10405E000DF0BAEC0DF0BAEC0DF0BAEC0DF0BAECC6
:10406E000DF0BAEC0DF0BAEC0DF0BAEC0DF0BAECB6
:10407E000DF0BAEC0DF089EC0EF089EC0EF089EC37
:10408E000EF08BD0BAEC0DF0BAEC0DF0BAEC0DF0E0
:10409E00BAEC0DF0BAEC0DF0BAEC0DF089EC0EF0B6
:1040AE0089EC0EF0BAEC0DF0BAEC0DF0BAEC0DF0A6
:1040BE00BAEC0DF0BAEC0DF089EC0EF089EC0EF0C6
:1040CE0089EC0EF0BAEC0DF0BAEC0DF0BAEC0DF086
:1040DE00BAEC0DF0BAEC0DF0BAEC0DF0BAEC0DF046
:1040EE0089EC0EF05AD0BAEC0DF0BAEC0DF0BAEC39
:1040FE000DF0BAEC0DF0BAEC0DF0BAEC0DF089EC57
:10410E000EF089EC0EF0BAEC0DF0BAEC0DF0BAEC44
:10411E000DF0BAEC0DF0BAEC0DF0BAEC0DF089EC36
:10412E000EF089EC0EF0BAEC0DF0BAEC0DF0BAEC24
:10413E000DF0BAEC0DF0BAEC0DF0BAEC0DF089EC16
:10414E000EF089EC0EF029D0FB51000AD8B4E1D55F
:10415E00FB51010AD8B40ED6FB51020AD8B43BD695
:10416E00FB51030AD8B468D6FB51040AD8B495D6CD
:10417E00FB51050AD8B4C2D6FB51060AD8B4EFD605
:10418E00FB51070AD8B41CD7FB51080AD8B449D73B
:10419E00FB51090AD8B476D7A6D703011C4B1D2BA9
:1041AE000201D351010F016E026A000E0222800E2F
:1041BE0003011D19006E800E0218005C02E1015011
:1041CE001C5DD8A09BD5090E0B6E1E0E0C6EE40E58
:1041DE000D6E0D2EFED70C2EFCD70B2EFAD700002F
:1041EE00000E0101821902E1000E811901E1F8D7DA
:1041FE00816B826B000E03011F1902E1010E1E1965
:10420E00D8A4A6D32B0E206F030E216F20C3E9FF77
:10421E0021C3EAFFEE50480A44E1030E2025E96E61
:10422E00000E2121EA6EEE50700A3BE1B10E040140
:10423E000A6F5A0E0B6F000E0C6F65EC05F0450EF3
:10424E0004010A6F580E0B6F000E0C6F65EC05F033
:10425E00D00E04010A6F590E0B6F000E0C6F65EC39
:10426E0005F0CD0E04010A6F570E0B6F000E0C6F8A
:10427E0065EC05F0370E04010A6F550E0B6F000E3C
:10428E000C6F65EC05F0260E04010A6F540E0B6FD1
:10429E00000E0C6F65EC05F0B3EC04F00301206B1F
:1042AE00216B20C3E9FF21C3EAFFEE50550A40E11E
:1042BE00130E2025E96E000E2121EA6EEE50230A20
:1042CE0037E1A40E04010A6F5B0E0B6F000E0C6F2C
:1042DE0065EC05F02B0E04010A6F030E0B6F99ECC3
:1042EE0003F0B3EC04F07CEC0AF0010E0301FD6F59
:1042FE00FEEC10F011C314F415EC01F000C0D3F273
:10430E0013C314F415EC01F000C000F3FFC214F453
:10431E0015EC01F000C012F318C314F415EC01F003
:10432E0000C0FEF2070E0201E7170301206B216B9E
:10433E0020C3E9FF21C3EAFFEE504D0A3DE1010E15
:10434E002025E96E000E2121EA6EEE503D0A34E181
:10435E00020E2025E96E000E2121EA6EEE50310A82
:10436E000AE0020E2025E96E000E2121EA6EEE50C3
:10437E00320A01E021D0020E2025E96E000E212125
:10438E00EA6EEECF16F3000E176F000E176F300E9B
:10439E00165D1B6FF00E04010A6F5B0E0B6F000EA5
:1043AE000C6F65EC05F016C31CF4ACEC00F0B3EC2E
:1043BE0004F00301206B216B20C3E9FF21C3EAFF48
:1043CE00EE50500AD8A49CD1010E2025E96E000EA5
:1043DE002121EA6EEE504C0AD8A492D1020E20256D
:1043EE00E96E000E2121EA6EEE504D0AD8A488D156
:1043FE00030E2025E96E000E2121EA6EEE503D0AD5
:10440E00D8A47ED12B0E04010A6F030E0B6F1CEC89
:10441E0004F0800E0118026E800E025C02E1090E9D
:10442E00005CD8A06DD1920E0A6F5C0E0B6F000E61
:10443E000C6F65EC05F020C30AF421C30BF499EC64
:10444E0003F0060E03012025E16E000E2121E26E1F
:10445E00E66A090E2025E16E000E2121E26EE66A63
:10446E00040E2025E96E000E2121EA6EEECF14F423
:10447E0041EC03F000C0FBF3050E03012025E96EAD
:10448E00000E2121EA6EEECF14F441EC03F0005041
:10449E000301FB27FC6B000EFC23070E2025E96EA3
:1044AE00000E2121EA6EEECF14F441EC03F0005021
:1044BE000301FB27000EFC23080E2025E96E000EDB
:1044CE002121EA6EEECF14F441EC03F0005003010B
:1044DE00FB27000EFC23FBC314F3FCC315F3040EE1
:1044EE002025E96E000E2121EA6E300EEE5C006E84
:1044FE00016A000E015A0A0E046E000E056EBAEC29
:10450E0001F0050E2025D96E000E2121DA6EDE5047
:10451E0000240101706F000E0120716F300E705F6C
:10452E00000E715B070E03012025E96E000E21219E
:10453E00EA6E300EEE5C006E016A000E015A0A0E33
:10454E00046E000E056EBAEC01F0080E2025D96E31
:10455E00000E2121DA6EDE5000240101896F000E5B
:10456E0001208A6F300E895F000E8A5B000E0301F8
:10457E00FC1902E1040EFB19D8A4B3D0000E006E94
:10458E0001017151005C02E170510908D8B0A9D047
:10459E00000E715D02E1180E705DD8B0A2D0000E53
:1045AE008A5D02E1000E895DD8A09BD0000E8A5D67
:1045BE0002E10A0E895DD8B094D070C1D3F071C1FA
:1045CE00D4F0040E03012025E96E000E2121EA6EBF
:1045DE00EECF24F3840EFD6F000EFE6F24C3FFF3A7
:1045EE0080EC11F0050E03012025E96E000E21214D
:1045FE00EA6EEECF24F3850EFD6F000EFE6F24C320
:10460E00FFF380EC11F0030E0B6E080E0C6E770E9E
:10461E000D6E0D2EFED70C2EFCD70B2EFAD789C1A0
:10462E00D1F08AC1D2F0070E03012025E96E000EEB
:10463E002121EA6EEECF24F3870EFD6F000EFE6F82
:10464E0024C3FFF380EC11F0030E0B6E080E0C6EFC
:10465E00770E0D6E0D2EFED70C2EFCD70B2EFAD725
:10466E00080E03012025E96E000E2121EA6EEECF21
:10467E0024F3880EFD6F000EFE6F24C3FFF380EC53
:10468E0011F0030E0B6E080E0C6E770E0D6E0D2EC6
:10469E00FED70C2EFCD70B2EFAD7D80E04010A6FBC
:1046AE005B0E0B6F000E0C6F65EC05F0530E0201E6
:1046BE00516F020E526F800E0401016F000E026FD9
:1046CE0051C203F452C204F4CDEC0CF051C20AF400
:1046DE0052C20BF499EC03F0B3EC04F0010E1F6E12
:1046EE000AD0080E04010A6F570E0B6F000E0C6FE6
:1046FE0065EC05F01F6AB3EC04F00301206B216B2F
:10470E0020C3E9FF21C3EAFFEE504C0AD8A420D102
:10471E000301010E2025E96E000E2121EA6EEE50F6
:10472E00750AD8A415D1020E2025E96E000E21219E
:10473E00EA6EEE506D0AD8A40BD1030E2025E96E59
:10474E00000E2121EA6EEE503D0AD8A401D12B0EA7
:10475E0004010A6F030E0B6F99EC03F0090E1C6F28
:10476E00ACEC00F0070E04010A6F5C0E0B6F000E2E
:10477E000C6F65EC05F0D0C014F4000E0401156F3B
:10478E00AB0E166F030E176FF8EC02F0AB0E0A6F3E
:10479E00030E0B6F99EC03F0090E1C6FACEC00F0DE
:1047AE00040E03012025E96E000E2121EA6EEECFE4
:1047BE0014F441EC03F000C0FBF3050E03012025B9
:1047CE00E96E000E2121EA6EEECF14F441EC03F0F7
:1047DE0000500301FB27FC6B000EFC23FBC314F3FC
:1047EE00FCC315F3040E2025E96E000E2121EA6E9E
:1047FE00300EEE5C006E016A000E015A0A0E046E57
:10480E00000E056EBAEC01F0050E2025D96E000ED5
:10481E002121DA6EDE5000240101706F000E01209E
:10482E00716F300E705F000E715B000E0301FC198C
:10483E0002E1020EFB19D8A47FD0000E0101715DBA
:10484E0002E1000E705D78E3000E715D02E10B0E69
:10485E00705D72E20F0E70150001D06F740E0301C1
:10486E00FD6F000EFE6F0A0E046E000E056E70C117
:10487E0000F071C101F0E1EC00F0300E0024FF6F8A
:10488E0080EC11F0030E0B6E080E0C6E770E0D6E93
:10489E000D2EFED70C2EFCD70B2EFAD7750E03015C
:1048AE00FD6F000EFE6F0A0E046E000E056E70C1D7
:1048BE0000F071C101F0E1EC00F008C000F009C099
:1048CE0001F0300E0024FF6F80EC11F0030E0B6E22
:1048DE00080E0C6E770E0D6E0D2EFED70C2EFCD71D
:1048EE000B2EFAD70A0E0401146FD0C015F4D0C0E7
:1048FE0016F4D0C017F4D0C018F4E2EC01F08A0E12
:10490E0004010A6F5C0E0B6F000E0C6F65EC05F068
:10491E00700E0401016F000E026FAB0E036F030EDB
:10492E00046FCDEC0CF0AB0E0A6F030E0B6F99EC0F
:10493E0003F0B3EC04F009D0A00E04010A6F570E79
:10494E000B6F000E0C6F65EC05F00301206B216BF5
:06495E0074EF1AF0FFD710
:105CFA0010EE19F0570E006E020E016E640EF66E6B
:0E5D0A00510EF76E000EF86E20EC08F012003D
:1049640000000000000000001010101010001000E3
:10497400242424000000000024247E247E24240017
:10498400183E403C027C1800006264081026460071
:10499400304830568888760010102000000000004F
:1049A400102040404020100020100808081020006B
:1049B400004438FE384400000010107C1010000041
:1049C40000000000001010200000007E0000000025
:1049D4000000000000101000000204081020400035
:1049E4003C42464A52623C001030501010107C0089
:1049F4003C42020C30427E003C42021C02423C001B
:104A040008182848FE081C007E407C0202423C0034
:104A14001C20407C42423C007E42040810101000DE
:104A24003C42423C42423C003C42423E020438008A
:104A340000101000001010000010100000101020D2
:104A4400081020402010080000007E00007E0000B6
:104A540010080402040810003C4202040800080084
:104A64003C425E525E403C00182442427E42420078
:104A74007C22223C22227C001C22404040221C003A
:104A840078242222222478007E22283828227E00BC
:104A94007E222838282070001C2240404E221E000E
:104AA4004242427E42424200381010101010380038
:104AB4000E0404044444380062242830282463008B
:104AC4007020202020227E0063554941414141004D
:104AD40062524A46424242003C42424242423C0006
:104AE4007C22223C202070003C4242424A3C03008B
:104AF4007C22223C282472003C42403C02423C007E
:104B04007F49080808081C004242424242423C00D5
:104B1400414141412214080041414149494936007B
:104B240041221408142241004122140808081C00E0
:104B34007F42040810217F007840404040407800C4
:104B4400804020100804020078080808080878004B
:104B5400102844820000000000000000000000FF54
:104B6400101008000000000000003C023E423F001C
:104B74006020202E31312E0000003C4240423C0097
:104B84000602023A46463B0000003C427E403C009E
:104B94000C1210381010380000003D42423E027CD6
:104BA40060202C32222262001000301010103800D5
:104BB400020006020242423C6020242830282600DB
:104BC400301010101010380000007649494949008F
:104BD40000005C624242420000003C4242423C000F
:104BE40000006C32322C20700000364C4C34040E21
:104BF40000006C322220700000003E403C027C0029
:104C040010107C1010120C000000424242463A0080
:104C1400000041412214080000004149494936007E
:104C2400000044281028440000004242423E027C16
:104C340000007C0810207C000C10106010100C0088
:104C4400101010001010100030080806080830007A
:104C5400324C0000000000001C14141C0000000072
:104C64003C4240423C0C023C0044004444443E006C
:104C74000C003C427E403C003C4238043C443E0034
:104C8400420038043C443E00300038043C443E00BA
:104C9400705077040404040700003C40403C061CA8
:104CA4003C423C427E403C0042003C427E403C0050
:104CB40030003C427E403C002400180808081C00D8
:104CC4007C823010101038003000180808081C00CE
:104CD400421824427E4242001818003C427E4200A0
:104CE4000C007C2038207C000000330C3F443B0047
:104CF4001F24447F444447001824003C42423C00A3
:104D04000042003C42423C002010003C42423C0035
:104D14001824004242423C002010004242423C001F
:104D240000420042423E023C4218244242241800FF
:104D34004200424242423C0008083E40403E0808CD
:104D44001824207020427C0044287C107C10100021
:104D5400F84C78444F4445E61C12107C10109060C7
:104D64000C0038043C443E000C00180808081C00E1
:104D74000408003C42423C000004084242423C0019
:104D8400324C007C42424200324C0062524A46009D
:104D94003C44443E007E000038444438007C00001B
:104DA4001000102040423C000000007E4040000003
:104DB4000000007E0202000042C448F629438C1F12
:104DC40042C44AF62A5F820200100010101010003C
:104DD4000012244824120000004824122448000031
:104DE400228822882288228855AA55AA55AA55AA1B
:104DF400DB77DBEEDB77DBEE1010101010101010F9
:104E040010101010F01010101010F010F0101010FE
:104E140014141414F414141400000000FC141414D6
:104E24000000F010F01010101414F404F41414140E
:104E340014141414141414140000FC04F41414149E
:104E44001414F404FC00000014141414FC000000F6
:104E54001010F010F000000000000000F01010101E
:104E6400101010101F00000010101010FF000000A0
:104E740000000000FF101010101010101F10101070
:104E840000000000FF00000010101010FF101010B0
:104E940010101F101F1010101414141417141414CD
:104EA400141417101F00000000001F10171414140E
:104EB4001414F700FF0000000000FF00F71414149E
:104EC40014141710171414140000FF00FF0000003E
:104ED4001414F700F71414141010FF00FF0000005E
:104EE40014141414FF0000000000FF00FF10101041
:104EF40000000000FF141414141414141F00000004
:104F040010101F101F00000000001F101F101010B1
:104F1400000000001F14141414141414FF141414A7
:104F24001010FF10FF10101010101010F0000000EF
:104F3400000000001F101010FFFFFFFFFFFFFFFF26
:104F440000000000FFFFFFFFF0F0F0F0F0F0F0F0E1
:104F54000F0F0F0F0F0F0F0FFFFFFFFF00000000D9
:104F64000000314A444A3100003C427C427C4040CB
:104F7400007E424040404000003F5414141414008A
:104F84007E42201820427E0000003E4848483000FF
:104F9400004444447A40408000334C080808080028
:104FA4007C1038444438107C1824427E4224180073
:104FB40018244242242466001C20183C42423C002F
:104FC400006295899562000002043C4A523C40808C
:104FD4000C10203C20100C003C4242424242420051
:104FE400007E007E007E000010107C1010007C000B
:104FF4001008040810007E000810201008007E002D
:105004000C1212101010101010101010109090604C
:105014001818007E0018180000324C00324C0000B2
:10502400304848300000000000000018180000005C
:1050340000000000180000000F08080808C828181D
:1050440078444444440000003048102078000000B4
:1050540000003C3C3C3C000000000000000000005C
:10506400000000000000000000000000000000003C
:10507400000000000000000000000000000000002C
:10508400000000000000000000000000000000001C
:10509400000000000000000000000000000000000C
:1050A40000000000000000000000000000000000FC
:1050B40000000000000000000000000000000000EC
:1050C40000000000000000000000000000000000DC
:1050D40000000000000000000000000000000000CC
:1050E40000000000000000000000000000000000BC
:1050F40000000000000000000000000000000000AC
:10510400000000000000000000000000000000009B
:10511400000000000000000000000000000000008B
:10512400000000000000000000000000000000007B
:10513400000000000000000000000000000000006B
:10514400000000000000000000000000000000005B
:10515400000000000000000000000000000000004B
:02516400000049
:02516600000047
:02516800000045
:01516A000044
:08516B0000808000008080003C
:105173000E1111131519110E040C14040404041F49
:105183000E1101070C18111F0E1101070101110E59
:10519300030509111F0101011F10101F0101190E41
:1051A3000F18101E1111110E1F110306080808080D
:1051B3000E11111F1111110E1F11111F0101011EDB
:1051C30070888898A8C888702060A020202020F8C4
:1051D3007088083860C088F87088083808088870B4
:1051E30018284888F8080808F88080F80808C87064
:1051F30078C080F088888870F888183020202020B4
:10520300708888F888888870F88888F8080808F013
:0852130000010100000101008F
:01521B000092
:02521C00080088
:02521E00150079
:10522000635A00845400BB5200AE5300365300E072
:1052300054008655002B5B001D5600D35500DE58E8
:01524000006D
:045241000000000069
:08524500705077040404040713
:08524D00000000000000808059
:0952550030302F30302F303000D2
:10525E00AE5C00B55C00BC5C00125C00995C003A70
:08526E005C00725C00265C008C
:10527600825C00605C00695C00C95C00A75C00EAB7
:105286005C00C35C004E5C00D55C00FC5B00575CB8
:07529600001C5C00305C000D
:09529D0030303A30303A30300074
:0852A6000000000000000101FE
:0852AE000000007C000000007C
:0152B60000F7
:0452B70000000000F3
:1052BB002050726F6A6574203A20486F726C6F676A
:1052CB00655F56345F474159415F31384632364B43
:1052DB0032325F345F4D6174726963653878385F61
:1052EB00485F4761756368655F416E6E6561755FA9
:1052FB0036306C6564735F5247425F446174655F1F
:10530B006A6F75725F48484D4E5F54656D705F41B3
:10531B006C7465726E6565735F323032305F303737
:0B532B0032352E6D637070690D0A00B2
:1053360020454570726F6D203A20486F726C6F671A
:10534600655F565F5370656369616C655F313846AA
:1053560032364B32325F345F4D6174726963653841
:1053660078385F485F416E6E6561755F36306C6593
:1053760064735F5247425F446174655F6A6F75721A
:105386005F48484D4E5F54656D705F416C74657241
:105396006E6565735F323032305F454570726F6D92
:0853A6002E696865780D0A000C
:1053AE0020536F75726365203A20486F726C6F6779
:1053BE00655F56345F474159415F31384632364B4F
:1053CE0032325F345F4D6174726963653878385F6D
:1053DE00485F4761756368655F416E6E6561755FB5
:1053EE0036306C6564735F5247425F446174655F2B
:1053FE006A6F75725F48484D4E5F54656D705F41C0
:10540E006C7465726E6565735F323032305F303743
:08541E0032352E63200D0A0057
:1054260020434F52313D2B303335302020636F728D
:1054360072656374696F6E2074656D702E204453B7
:10544600313842323020656E20312F313030656D73
:105456002064652064656772200D0A20434F52312F
:105466003D2B30353020286C696D69746573202DAD
:0E54760033303020E0202B333030290D0A0077
:10548400204469726563746F7279203A20433A5CF0
:105494005F4D696B726F435C5F4D657350726F6AE9
:1054A4006574735F4D696B726F435C5F486F726CB8
:1054B4006F67655F416E6E6561755F36306C6564FC
:1054C400735F31384632364B32325F476179615F00
:0C54D4004D6F7274696D6572200D0A0046
:1054E0002050696E2052423320706F7572206368BD
:1054F0006F697820636F6E6E656374696F6E2047A5
:1055000061756368653D30206F752044726F697402
:10551000653D31206465732034204D617472696388
:105520006573203878382048204D4158373132395A
:0755300020434D530D0A005A
:105537002047616D6520506C616765204C756D690A
:105547006E6F73697465204D696E696D616C652056
:10555700504C4D3D32313B30383C43523E0D0A20D2
:105567004D696E696D6120656E74726520203231F8
:0F5577004830302065742030384830300D0A003D
:10558600204C696169736F6E20426C7565546F6F4C
:105596007468202F205465726D696E616C20706F7F
:1055A6007572206469616C6F677565206574205635
:1055B60069737520206465726F756C656D656E74B0
:0D55C6002070726F6772616D6D650D0A00D7
:1055D30020417574726573203A2054696E795F5265
:1055E30054435F4453333233315F666F725F4149D3
:1055F300325F323032305F30372E63202020466FE7
:105603006E7465203A205448494E5F53535F3230DD
:0A56130032305F30372E680D0A00B8
:10561D00205350492057533238313220626974205B
:10562D0062616E6720706F757220416E6E65617577
:10563D0020657420535049206269742062616E6741
:10564D0020706F7572204D4158373231390D0A0077
:10565D00204269742042616E6720536F6674205337
:10566D00504920205243323D436C6B202C52433124
:10567D003D446F757420205243303D4353202D3EE1
:0C568D00204D4178373231393A0D0A00C7
:1056990020553A32343B30383B31373B31383B3394
:1056A900363B3034232020706F7572204A6575644B
:1056B9006920323420416F7574203230313720200F
:0A56C90031384833360D0A0D0A008F
:1056D3000D0A2052617070656C20666F726D617483
:1056E30020646520636465203A2022553B4A4A3B87
:1056F3004D4D3B41413B48483B4D4D3B6A443B2369
:0557030022200D0A0048
:105708002042414420504C4D2076616C75657321D0
:10571800206D7573742062652066726F6D205B3131
:1057280030202E2E2032335D20746F205B30202EE7
:045738002E395D00A9
:10573C00205465737420696E746572727570742070
:10574C0054696D6572312020323020782031303030
:10575C00206D73656320736F6974203273656320E9
:03576C000D0A0023
:10576F00204465636F6D70696C6520636869666658
:10577F00726520472026204420617665632073657B
:10578F00706172617465757273204420657420476F
:01579F000009
:1057A00020424144204C756D2076616C7565202146
:1057B000206D757374206265206265747765656E0F
:0D57C00020303020616E642031300D0A0071
:1057CD00204475726565204D656C6F6469653A445A
:1057DD004D3D30333C43523E67616D6D6520322047
:0857ED00E0203230730D0A00C8
:1057F50020456E74726565205072655F544553543B
:10580500204E4F4E20206163746976E96520285249
:0858150041323D30290D0A006B
:10581D0020496E697420496E7465727275707420BA
:10582D005242302C2073796E6368726F2031487A42
:08583D0020525443200D0A0023
:1058450020525443205570646174653A20553B31AC
:10585500343B30353B31383B31353B33363B3032E9
:08586500233C43523E0D0A00F2
:10586D0020526563757065726174696F6E20646135
:10587D0074617320656E2045656570726F6D205083
:06588D004943200D0A0052
:1058930020456E74726565205072655F544553549C
:1058A3002044E9736163746976E9652028524132C3
:0658B3003D30290D0A0042
:1058B90020496E697420496E74657272757074201E
:1058C90054696D6572312020262055415254205269
:0558D90058200D0A003B
:1058DE002041766563204D65737572652054656D44
:1058EE00706572617475726520445331384232307E
:0458FE00200D0A006F
:105902002043686F697820636F74E920436F6E6E7D
:10591200656374696F6E204D415452494345204876
:0459220020E0200061
:10592600205072655F5465737420506172636F75A1
:10593600727320646573203630206C656473202092
:035946000D0A0047
:1059490020456E74726565205072655F54455354E5
:10595900206163746976E96520285241323D312915
:035969000D0A0024
:10596C000D0A45727265757220737572204A6F75D7
:10597C00722053656D61696E65206A532E204F4B02
:03598C000D0A0001
:10598F00202E2E2E2057616974696E67204B657922
:10599F00626F61726420546F75636820666F722046
:0259AF003C00BA
:1059B10020546573742043646520444F75742052EC
:0F59C1004335202E2E20656E2041534D0D0A00D8
:1059D000203134204D616920323031382030322876
:0F59E0004C756E6469292031354833360D0A0045
:1059EF002054656D706572617475726520696E748F
:0F59FF0065726E6520445333323331203D2000F2
:105A0E0045637269747572652064616E73204453C8
:0D5A1E00333233312E2E2E204F4B0D0A0057
:105A2B00696E69742076616C65757273205254438C
:0D5A3B002070617220646566617574200042
:105A48002041637469766520736F727469652053A9
:0B5A580051573D31487A3A200D0A00FA
:105A6300204D696B726F6320372E362E302031380C
:0A5A73004632364B3232200D0A0095
:105A7D00205465737420536F6E6465204F57532007
:0A5A8D00445331384232300D0A0054
:105A97000D0A2052415A20616E6E656175203630BD
:0A5AA700206C65647320200D0A00D6
:105AB1000D0A2048656C70203A2048656C703C43A3
:075AC100523E20200D0A00F7
:105AC80020496E6974205254432044533332333191
:055AD8003A200D0A0058
:105ADD0020436C6561722034204D61747269636579
:045AED00200D0A007E
:105AF10020496E69742034206D6174726963657325
:045B0100200D0A0069
:105B05002050726573656E746174696F6E203A20FA
:035B15000D0A0076
:105B180044757265652052415A20616E6E656175E3
:035B28003D20001D
:105B2B0020416C696D203D332E36565F6D696E6971
:035B3B000D0A0050
:105B3E00204D657375726520445331384232303DC5
:025B4E00200035
:105B500044757265652074656D702035306D533DF8
:025B6000200023
:105B62002052652D4C656374757265205254432032
:015B72000032
:105B730045724C754D614D654A655665536144697F
:015B83000021
:105B8400303132333435363738394142434445466F
:105B94002046616D696C7920436F6465203A20006A
:0E5BA40052544320557064617465203A20000D
:0D5BB20044524F49544520285242333D00D3
:0D5BBF0047415543484520285242333D00E0
:0C5BCC002056616C69645F504C4D3D0038
:0C5BD800204E657720504C4D203A2000F4
:0C5BE40020782032356D53203E0D0A0061
:0C5BF0004E6577204D6F6465203D20005D
:0B5BFC0053657074656D6272652000D7
:0B5C0700204F6C64204C756D3D2000A8
:0A5C12004D6572637265646920003D
:0A5C1C004E6F76656D627265200020
:0A5C260044696D616E63686520003B
:0A5C3000446563656D627265200033
:0A5C3A0056656E647265646920000F
:0A5C44002074696D6520697320006B
:095C4E004A75696C6C6574200054
:095C57004F63746F627265200056
:095C60004A616E7669657220004C
:095C69004665767269657220003F
:085C720053616D6564692000B7
:085C7A0020204352433D2000AD
:085C8200657272657572200065
:085C8A00204E6577203D20004B
:075C9200436465203A200085
:075C99004A657564692000F3
:075CA000204944313D2000C2
:075CA700417672696C2000D8
:075CAE004572726F722000C5
:075CB5004C756E64692000CC
:075CBC004D617264692000D4
:065CC3004A75696E200025
:065CC9004D617273200022
:065CCF0054496E203D0067
:065CD500416F7574200010
:055CDB00B04320200091
:055CE000B0432020008C
:055CE500B5530D0A009B
:055CEA004D616920007E
:055CEF00B5530D0A0091
:035CF4002020006D
:035CF7002020006A
:020000040030CA
:0D00010038183CFFBF81FF0FC00FE00F401B
:0200000400F00A
:10000000486F726C6F676520416E6E656175202068
:100010003630206C6564732052474220202B2034F8
:10002000204D617472696365732038783820480DFB
:100030000A7665722032303230303731320D0A00A4
:10004000FFFFFFFFFFFFFFFFFFFFFFFFFFFFFFFFC0
:10005000FFFFFFFFFFFFFFFFFFFFFFFFFFFFFFFFB0
:10006000FFFFFFFFFFFFFFFFFFFFFFFFFFFFFFFFA0
:100070004C756D3D30310D0A00FFFFFFFFFFFFFFA4
:10008000504C4D3D32313A30350D0A00FFFFFFFF35
:1000900053706565643D39300D0A00FFFFFFFFFFB7
:1000A000434F52313D2B3031300D0A00FFFFFFFF2F
:1000B000FFFFFFFFFFFFFFFFFFFFFFFFFFFFFFFF50
:1000C000FFFFFFFFFFFFFFFFFFFFFFFFFFFFFFFF40
:1000D000FFFFFFFFFFFFFFFFFFFFFFFFFFFFFFFF30
:1000E000FFFFFFFFFFFFFFFFFFFFFFFFFFFFFFFF20
:00000001FF
